:1000000003C5000039C5000037C5000035C5000034
:1000100033C5000031C500002FC500002DC500000C
:100020002BC5000029C500000C9468320C94503395
:100030000C941D3221C500001FC500001DC5000025
:100040001BC5000019C5000017C5000015C500003C
:1000500013C500000C9444320FC500000DC500000C
:100060000BC5000009C5000007C5000005C500005C
:1000700003C5000001C50000FFC40000FDC400006E
:10008000FBC40000F9C40000F7C40000F5C4000080
:10009000F3C40000F1C40000EFC40000EDC4000090
:1000A000EBC40000E9C40000E7C400000501090238
:1000B000A10185020901A1000509190129081500FE
:1000C0002501950875018102050109300931158165
:1000D000257F95027508810609381581257F9501D0
:1000E00075088106050C0A38021581257F95017572
:1000F000088106C0C005010980A101850319012AF4
:10010000B700150126B700950175108100C0050CD8
:100110000901A101850419012AA002150126A002E6
:10012000950175108100C005010906A1018506052C
:100130000719E029E71500250195087501810205D9
:1001400007190029EF1500250195F07501810205B9
:10015000081901290595057501910295017503910D
:1001600001C00660FF0961A1010962150026FF00B8
:100170009520750881020963150026FF00952075FA
:10018000089102C005010906A101050719E029E748
:1001900015002501950875018102950175088101F9
:1001A0000507190029FF150026FF0095067508812F
:1001B000000508190129051500250195057501910E
:1001C00002950175039101C00000000000000000CD
:1001D000000000000000000000000000000000001F
:1001E0000000000000000000000000007E0F00D4AE
:1001F000FFFFFFC7000000780000000000000000C3
:100200002A2B280000000000000000000000000071
:1002100000000029000000002C1E3420212224347C
:100220002627252E362D3738271E1F20212223244E
:1002300025263333362E37381F0405060708090AEA
:100240000B0C0D0E0F101112131415161718191A86
:100250001B1C1D2F3130232D350405060708090A04
:100260000B0C0D0E0F101112131415161718191A66
:100270001B1C1D2F3130354C09025B00030100A00F
:10028000FA09040000010301010009211101000124
:10029000224400070581030800010904010002034C
:1002A000000000092111010001222200070582033C
:1002B00020000107050303200001090402000103D7
:1002C00000000009211101000122B6000705840386
:1002D000200001120100020000000845585256019A
:1002E00000010203011C037600690061006C003A02
:1002F00000660036003400630032006200330063A1
:100300000000001603560061006C006F00720020B0
:1003100000520065007600310000000C03580065B3
:10032000006C007500730000000403090429003507
:10033000021E001F002000210022002300240025AF
:1003400000260027002D002E004C004B002B00142F
:10035000001A000800150017001C0018000C0012FD
:100360000013002F00300031004E00390004001649
:1003700000070009000A000B000D000E000F0033FB
:1003800000340028002A000000E1001D001B0006C8
:100390000019000500050011001000360037003874
:1003A00000E500E7000000E0000000E20000002C93
:1003B00000215200002C000000E60000000000E4D4
:1003C000000000207801003A003B003C003D003E68
:1003D000003F00400041004200430044004500014E
:1003E000002178010001000100010001000100016D
:1003F00000010001000100010001000100010000F6
:100400007C01000100010001000100010001000168
:1004100000010001000100010001000100000001D5
:1004200000010001000100010001000100010001C4
:1004300000010001000100010001000000010000B6
:1004400000010000000100010000000100000001A7
:100450000000000000010000000100010001000197
:100460000001000100010001000100010001000184
:100470000001000100010001000100010001000174
:100480000001000100010001000100010001000164
:100490000001000100010001000100010001000154
:1004A0000001000100010001000100010001000144
:1004B0000001000000010001000100010001000135
:1004C0000001000100010001000100010001000124
:1004D0000000000100000001000000010001000018
:1004E0000001000000010000000000010000000108
:1004F00000010001000100010001000100010001F4
:1005000000010001000100010001000100010001E3
:1005100000010001000100010001000100010001D3
:1005200000010001000100010001000100010001C3
:1005300000010001000100010001000100010001B3
:1005400000010001000100010000000100010001A4
:100550000001000100010001000100010001000193
:100560000001000100010000000100000001000086
:100570000001000100000001000000010000000077
:1005800000010000002223252628292A2C2D2F30A7
:1005900032333536383A3B3D3E4042434547494A7F
:1005A0004C4E5051535557595A5C5E6062646668B0
:1005B000696B6D6F71737577797B7D7F81838587BB
:1005C000898A8C8E90929496989A9C9E9FA1A3A5BE
:1005D000A7A8AAACAEAFB1B3B4B6B8B9BBBCBEBFE6
:1005E000C1C2C3C5C6C7C9CACBCCCDCED0D1D2D269
:1005F000D3D4D5D6D7D7D8D9D9DADADBDBDBDCDC74
:10060000DCDCDCDDDDDDDDDCDCDCDCDCDBDBDBDA2B
:10061000DAD9D9D8D7D7D6D5D4D3D2D2D1D0CECD96
:10062000CCCBCAC9C7C6C5C3C2C1BFBEBCBBB9B8A3
:10063000B6B4B3B1AFAEACAAA8A7A5A3A19F9E9C28
:100640009A98969492908E8C8A89878583817F7DF3
:100650007B79777573716F6D6B6968666462605ED4
:100660005C5A5957555351504E4C4A49474543429D
:10067000403E3D3B3A3836353332302F2D2C2A2937
:100680002826252322FFAA7F5540000101010101F0
:10069000010101010202020202020202020303033B
:1006A000030303030304040404040404050505050B
:1006B00005060606060607070707070808080809CB
:1006C0000909090A0A0A0B0B0B0C0C0C0D0D0D0E77
:1006D0000E0E0F0F0F10101111111212131314140C
:1006E000151516161717181819191A1A1B1B1C1D81
:1006F0001D1E1E1F202021222223242425262627DA
:100700002829292A2B2C2D2D2E2F3031323233340B
:1007100035363738393A3B3C3D3E3F404142434411
:1007200045464748494A4C4D4E4F505153545556F3
:1007300058595A5B5D5E5F616264656668696B6C9F
:100740006D6F7072737577787A7B7D7E808283851A
:1007500087888A8C8E8F91939596989A9C9EA0A25A
:10076000A3A5A7A9ABADAFB1B3B5B7BABCBEC0C264
:10077000C4C6C9CBCDCFD1D4D6D8DBDDDFE2E4E728
:10078000E9EBEEF0F3F5F8FAFDFF1E0F0500047F2C
:100790003F1F643214643214783C1E1E140A05FD97
:1007A000377A585A000004E6D6B4460200210116F2
:1007B000000000742FE5A3E006B002265D003D882E
:1007C00089C65436C3174FE4E7DF56602461CCE195
:1007D000F809AE3065C85D2CE4DE3481BEF6FF4416
:1007E00019F9F21747136F6D8C014C4393C56026BE
:1007F000360955C9876A299ABBD05D1499F7A04F6D
:100800006C621EA053955567217221B89F039C8A84
:10081000911CE540DAE904CD6832DC7188ACE28EE7
:10082000C96822F3A0C8EB956BA6E43AE06591F4A1
:10083000622A95A0816531DC5F44D98F58292ACA84
:1008400098BA5FABED63BB10A16F78E4C17EFF384F
:10085000AA9DAD57526684A46CF2237D4C48F522C4
:10086000ED43B3C5FC4D9DFD0F5C89F9D7F56313CE
:10087000B1A4F54E0757C086D0E5247CE77371829A
:10088000B2ABDAA65EF0162680986FE81CA38761EB
:100890009B4CD980199F5A971FDB05629FB86A4A03
:1008A0003AAC68CE53FDEE9165950854C8BB1C1256
:1008B0003C0B4057122D4EC31E15A3081288F62B71
:1008C000560376E66CF3D4AF843A4E79A883B97AAE
:1008D0006BB6D2A5FDC3165733233E1EC73E5F97A6
:1008E000F46D467A974CBB5C89D2F233FDDAFE5741
:1008F0006309B95084E2352031608D39E08DED4DCA
:10090000E00A495BDE591055E23B9E1E8312B61287
:10091000A60E2ED9153B201EDA63B0969B5C0320F1
:100920003BF0265678A85FAB760B45451D0344F394
:10093000CD9761E6F95B031F2E592F834A69579BB8
:10094000F97740930C0BF8D103519D424E962FC678
:100950005232029F972E18C107EFD67BBEDD43DCD3
:100960005846D3FFAF3EA2CD76F2215BE8F58975FC
:100970007A340ACFE549E36490BABBD8101ADB1D7C
:1009800014A40E5616DC31700C7B0FE79568513AB3
:100990003D5757EEA92C9C4B1EC4D03A83A9A63EC6
:1009A00055B406C77ACE6DF342F2F285C0A0371275
:1009B000DD781AA38352DB1867F7758792ADD87973
:1009C00013D49BBAE2F0FDEC6C8CB675E444D1957F
:1009D000C4BCD35F9B330C81B7FA107DE607B1B678
:1009E000D62A1100000000DC0896DE76753076000D
:1009F00001C204B10D00000E77E3C7B1C467FB026A
:100A00000000000004595A0011241FBECFEFDAE0A5
:100A1000DEBFCDBF04B603FE18C08091A40590913F
:100A2000A505A091A605B091A7058730904BA740DA
:100A3000B04B59F41092A4051092A5051092A6058A
:100A40001092A705E0E0F8E3099525E0A6EEB1E0F5
:100A500001C01D92A43AB207E1F711E0A0E0B1E0B5
:100A6000E6E4FCE602C005900D92A63EB107D9F778
:100A70000E946C2A0C94A335C3CA9C01FB019A9571
:100A800081159F4120F5832F8170B32FB270AA2763
:100A9000732F74706627532F5870442734FF0DC08E
:100AA0008295807FAB2B09F08062672B09F0806410
:100AB000452B09F0806809950895AB2B09F08260F9
:100AC000672B09F08460452BB1F38860F4CF80E098
:100AD000F2CF982F92959F7024E0911102C020E0F0
:100AE000982F892F86958695811511F02E5F982F66
:100AF000892F8695820F08958093A005089580938D
:100B0000A105089521E030E001C0220F8A95EAF79F
:100B10008091A105822BF3CF21E030E0A90102C032
:100B2000440F551F8A95E2F7CA0180959091A1055F
:100B30008923E5CF292F953090F58F3080F590E00F
:100B40003FE0239F800D911D1124282F277041E045
:100B500001C0440F2A95EAF723E0969587952A95D8
:100B6000E1F7FC01EE0FFF1FE80FF91FEE5DFB4FF1
:100B700020E030E070E05191DF01CB01022E02C095
:100B8000969587950A94E2F781708195852784234D
:100B900085278E932F5F3F4F2330310561F70895EE
:100BA000292F953078F58F3068F590E03FE0239F4E
:100BB000800D911D1124682F677023E0969587950D
:100BC0002A95E1F7FC01EE0FFF1FE80FF91FEE5D1C
:100BD000FB4F40E050E080E0219130E0062E02C063
:100BE000369527950A94E2F721703327042E01C029
:100BF000220F0A94EAF7822B4F5F5F4F4330510573
:100C000059F7089580E008959091A10521E030E022
:100C1000F90101C0EE0F8A95EAF7D90102C0AA0FC7
:100C2000BB1F6A95E2F7EA2B01C0220F4A95EAF74B
:100C3000892F8E23E81303C0892F822B60CF209544
:100C4000822F8923FBCF8091D0039091CF039813FB
:100C500001C008958F5F8770FACF9091EC04809562
:100C600089238093EC04282F2770211110C0891745
:100C700071F09091A30592FF0AC08695869586959E
:100C80004BDF1092EC041092EE041092ED040895E4
:100C90009091E904982B9093E9040895982F9095EA
:100CA0008091E90489238093E90408958091E80400
:100CB000811531F01092E8041092F0041092EF04C4
:100CC0000895803E9105D9F1C8F48133910509F466
:100CD00082C048F48932910509F472C08A329105C4
:100CE00009F480C0089589339105E9F082389105AF
:100CF000D1F08533910509F45EC00895843E9105D5
:100D0000D9F148F4823E910539F1833E910549F1CC
:100D100081EE90E00895863E9105C9F1873E9105E8
:100D200009F43EC008952091A2052370211164C0EA
:100D30002091A30523FF14C089E290E0089520913B
:100D4000A20520FD45C03091A30530FF09C024FD58
:100D500024C083EE90E008952091A20522FDF7CFF4
:100D600008952091A20522FD44C03091A30530FDD5
:100D700043C024FFF5CF11C02091A30521FFF0CF80
:100D80008091A20584FD09C087EE90E0089520912E
:100D9000A20523FFE5CF24FFF7CF80E090E0089580
:100DA0002091A20523FD2BC03091A30531FFE1CF97
:100DB00084EE90E008952091A20525FFD1CFBCCF0D
:100DC0002091A20525FD1EC02091A30523FFC8CFB9
:100DD00089E390E008952091A20526FFC1CF8AE221
:100DE00090E008952091A20526FFBACF81E390E01C
:100DF000089582EE90E0089580EE90E0089586EEEA
:100E000090E0089585E390E008959091A20592FF07
:100E100010C041E0282F2471243009F040E031E077
:100E2000282F2871283009F030E0431711F02CE00A
:100E3000822793FF10C041E0282F2471243109F04C
:100E400040E031E0282F2871283109F030E04317C5
:100E500011F02CE082273091A30530FF10C051E043
:100E6000282F2171213009F050E041E0282F28710E
:100E7000283009F040E0541711F029E0822731FFB3
:100E800010C041E0282F2171213109F040E031E00C
:100E9000282F2871283109F030E0431711F029E09C
:100EA000822794FD877E08951F93CF93DF9309DFF8
:100EB000EC01811522E5920708F052C0811540E54A
:100EC000940708F0CDC0803E910520F58D3C91053A
:100ED00008F0A1C0883A910570F4853A910508F0B0
:100EE00097C081309105B9F10497813A910598F145
:100EF000C0E0D0E030C0885A91094B97C8F7C85A73
:100F0000D0E0CC0FDD1FC658DE4F0990D881C02D30
:100F1000D46421C0811550E49507B0F4C11580E276
:100F2000D80708F0B3C0C83ED105A8F0CE019A9505
:100F300081159F41E8F68D2F68DF182FCE01992784
:100F4000C0DEEC01D12B07C09927BBDECC27DF70B8
:100F5000C82BD92BD06ACE01DF91CF911F91089574
:100F6000803842E59407C8F5803652E5950708F0C9
:100F70005BC0C03482E5D807D0F4C03292E5D9070F
:100F800008F04BC08C2F8695869520E2829FC00189
:100F90001124C37021E030E0A90102C0440F551FA5
:100FA000CA95E2F7EA01C82BD92BDD68D4CF8C2F84
:100FB00086958695877050E2859FC0011124C37085
:100FC00021E030E0A90102C0440F551FCA95E2F7A5
:100FD000EA01C82BD92BDC68BECF803C52E59507CF
:100FE00058F48F71C03AD245A0F590E0982F882729
:100FF000EC01C46FD06AAFCF805C9245809708F057
:1010000077CFDC2FCC27CC27DF71C06FD06AA3CF7E
:10101000A497D064A0CFD0659ECFCF71D0E0DC2F55
:10102000CC27C16FD06A97CF86958695877020E2CE
:10103000829FC0011124C37021E030E0A90102C0E9
:10104000440F551FCA95E2F7EA01C82BD92BDA687D
:1010500082CFDBDEC82FD0E0DC2FCC27D0627BCF65
:101060008F71D3DE93E0CC0FDD1F9A95E1F7CC278B
:10107000DF70282F30E084FF05C050E1859F90018C
:1010800011243327C22BD32BD06965CF8D2F8F71BD
:10109000BCDE182FCE01992714DEEC01D12BDECF58
:1010A00080E00895F894E82FE295EF70F0E041A118
:1010B0008F7021E030E0B90102C0660F771F8A957A
:1010C000E2F7CB01962F9095942391A392A1892BBF
:1010D00082A3789408950895CF92DF92EF92FF92C1
:1010E0001F93CF93DF93172FE82FF0E0E657F94FC8
:1010F00071110CC0E4918E2F7E2F6E2FDF91CF9156
:101100001F91FF90EF90DF90CF900895E62EF12C85
:10111000C72ED12CF491EF2F86E0689F9001112407
:10112000CFEFD0E0C901BE010E94B433AB01EE0C99
:10113000FF1C65E5649FC001659F900D1124E81AAE
:10114000F90A6E2D660F6E0D7E01EC18FD08FE9DEE
:10115000D001FF9DB00D11248B2F169F700111241B
:10116000EF2CFF246E01CE18DF087601FE9D600192
:10117000FF9DD00C11247E01E61AF108B701169FDD
:101180007001179FF00C1124EF2CFF24CE19DF09FA
:10119000FC9F7001FD9FF00C11247F2D4330510501
:1011A000C1F02C3F334058F441305105B1F042308A
:1011B000510509F0A2CFEB2F8F2D7F2F9ECF44300A
:1011C000510571F04630510509F497CF7B2F8D2DD5
:1011D00094CF7D2DEB2F8F2F90CF7F2FED2D8DCFA7
:1011E000EF2D7B2FF8CFCF93982F762F842FC22F00
:1011F000692F72DF472F282F8C2F90E04BD2CF9191
:1012000008958091DF04843060F48370846080935B
:10121000DF048091E204893C18F088EC8093E204BA
:1012200008958C3AB0F38370886AF1CFCF93DF933F
:101230008091DF0480FD0BC0C0E0D0E020E040E002
:1012400060E0CE0127D22196CC31D105B9F787D6FF
:10125000DF91CF910895FF920F931F93CF93DF9368
:10126000182F062FF42E8091DF0480FF0CC0C0E001
:10127000D0E02F2D402F612FCE010CD22196CC3102
:10128000D105B9F7D3DFCDB7DEB7E5E00C941D3457
:10129000CF93DF93EC012091E2049C81892F817030
:1012A00090FD822F692F627091FD622F492F44704B
:1012B00092FD422FD0DF8C8190E0019687709927B4
:1012C0008C83DF91CF910895982F762F842F2091D2
:1012D000DF0420FF0AC0493C08F088EC692FFCDEDF
:1012E000962F672F482F892FB6CF0895CF93DF937E
:1012F000EC01EFEDF4E0438162818C81E5DF8C81CC
:101300008F5F8C83DF91CF910895CF93DF93EC01B2
:10131000EC81F0E0EB57FA4F4491EFEDF4E062819D
:101320008181D2DF8C818F5F8C83DF91CF91089593
:10133000FF920F931F93CF93DF93EC01F12C00E00A
:1013400010E04091E204493C08F048EC8C8198019F
:101350006091E1048F0D47DF0F5F1F4F89E0F80EAA
:101360000C31110571F762DF8C819A8190FF07C003
:101370008F5F8C83CDB7DEB7E5E00C941D348150D0
:10138000F8CFEF92FF920F931F93CF93DF93FC015F
:101390008281FF24F39480FF02C0FF24FA94C0E00E
:1013A000D0E020E040E060E0CE0174D104E010E045
:1013B000E12C80916A038E0D8D31A4F16CE10E94C5
:1013C000A733892F082E001C00088C170D0691F4F6
:1013D0004091E2040403A0011124559547955595C9
:1013E0004795493C08F048EC9E016091E1048091EA
:1013F000E004F9DEEF0C01501040D9F62196CC3113
:10140000D10579F613DF80916A03F1E0FF120EC077
:10141000811591F0815080936A03CDB7DEB7E6E085
:101420000C941C3487FFCECF845ECCCF90E0019625
:10143000BE010E94C833EFCF8BE1EDCFCF93DF9396
:10144000C0E0D0E020E040E060E0CE0123D1219672
:10145000CC31D105B9F7C0E0D0E080916903082E06
:10146000001C0008C817D00574F180910601082EF1
:10147000001C00088C170D0634F14091E204493C31
:1014800008F048EC9E016091E1048091E004ABDE3D
:101490002196CC31D10509F7C9DE809105019091E3
:1014A0006903980F9093690320910601280F2093F8
:1014B0000601121614F49B311CF0819580930501EE
:1014C000DF91CF91089520E040E060E0CE01E2D0CE
:1014D000DFCFA6E0B0E0EFE6FAE00C94FE338D83B8
:1014E0009E83AD81BE811496FC912F2F30E0D901EF
:1014F0000E9494359B01AC010E9462356B017C0116
:1015000080E290E09C012F1B3109F901A5E5B0E0D4
:10151000A70196010E94623569837A838B839C833D
:101520009F01DF010E94E8339B010E94EE339B0183
:10153000AC012C0D3D1D4E1D5F1D69817A818B8193
:101540009C810E947235022F30E00A32B8F5C90141
:10155000880F991F820F931F95958795182F1095C7
:10156000E12CF12C85E5D82ED01A8D2DE1FC802FB1
:10157000412F193C08F048EC97016091E10433DEFB
:101580005FEFE51AF50A8CE1E816F10471F74EDE1B
:10159000AD81BE8114969C9181E0911519F0903235
:1015A00019F48FEF8093040180910401890FED817C
:1015B000FE8184832696E8E00C941A3485E590E059
:1015C000AC01421B530B9A01CA01880F991F820F6D
:1015D000931F97FFC1CF0196BFCF0F931F93CF9358
:1015E000DF93EC0120E030E06091E1048091E004C1
:1015F0009C8189010F5F1F4F2E30310554F49115E6
:1016000001F14091E204493C08F048ECECDD98011E
:10161000EBCF911116C04091E204493C08F048EC30
:10162000E2DD98010C311105F9F600DE8C8190E0C5
:101630000196817099278C83DF91CF911F910F9133
:10164000089540E0EDCF81152CE7920741F42091F9
:101650009C0330919D03232B11F480E090E00895CA
:10166000E7E5F4E080E090E068E378E24BE558E2FB
:101670002DEC38E277836683518740873387228752
:1016800097878687019670968830910599F7089517
:10169000209A0895FC01EE0FFF1FE80FF91FEF5C81
:1016A000FD4F61834083228308951092320510928A
:1016B0003105E1EFF4E08581811102C014821682C8
:1016C000379685E0E932F807B1F70895AC0130911B
:1016D000340560913305232F621301C00895822FD2
:1016E00090E0FC01EE0FFF1FE75DFA4F0190F081E3
:1016F000E02DE417F50791F467E0649FF001659F22
:10170000F00D1124EF50FB4F41E044832313E6CF4B
:101710000196837099278093340508950196282FA8
:101720002370DACF0F931F93CF9301E010E0082EC0
:1017300001C0000F0A94EAF7C091E7049C2F9023A0
:10174000911115C09091EC049695969596958913F4
:1017500006C01092EC041092EE041092ED04D2D95F
:10176000C027C093E704CF911F910F910895D4D95A
:10177000F7CF282F35EB2303C001112497FF04C0B6
:1017800080589109892F089580589F4FFBCF8091F1
:10179000420480FD14C081FD14C082FD16C08091FA
:1017A0004104811581F08E3180F420E5829FC001D3
:1017B00011246EE170E00E94C833862F089584E101
:1017C000089588E2089588E0089580E5089580915D
:1017D000420480FD17C081FD17C082FD19C08091B1
:1017E0004004811599F0883298F428E0829FC00166
:1017F000112468E270E00E94C8336115710551F050
:10180000862F089562E0FCCF64E0FACF61E0F8CF64
:1018100068E0F6CF81E00895FA01309709F0099564
:101820000895E091C503F091C603309739F0019017
:10183000F081E02D309711F00995089580E008952A
:10184000A3E0B0E0E6E2FCE00C9404349C0180915B
:101850002E0290912F0282179307B1F030932F023E
:1018600020932E02E091C503F091C603309761F0FA
:101870000084F185E02D309739F083E089833B8344
:101880002A83CE01019609952396E2E00C94203438
:10189000A3E0B0E0EEE4FCE00C9404349C01809101
:1018A0002C0290912D0282179307B1F030932D02F4
:1018B00020932C02E091C503F091C603309761F0AC
:1018C0000084F185E02D309739F084E089833B83F3
:1018D0002A83CE01019609952396E2E00C942034E8
:1018E00090912001913091F0AAEEB1E0EFEF90E0FD
:1018F0002D91821751F0EF3F19F4211101C0E92F0A
:101900009F5F9630A9F7EF3FC9F408959091A20523
:1019100097FFEACFE82FE695E695E695803FA8F792
:10192000F0E0E051FE4F877021E030E001C0220F6F
:101930008A95EAF78281822B828308950E2E000C0D
:10194000FF0BE851FE4FF8CF90912001913021F428
:101950009091A20597FD0CC0EAEEF1E091918913F8
:1019600002C0DF011E9251E0E03FF507B9F708958C
:10197000E82FE695E695E695803FC8F7F0E0E05160
:10198000FE4F877021E030E0A90102C0440F551FCF
:101990008A95E2F7CA01809592818923828308950E
:1019A00080911F0108952FB7F8948091280290919B
:1019B0002902A0912A02B0912B022FBF0895CF9344
:1019C000DF93C091E9048091EB04C82B8091E80477
:1019D0008115F1F0E8DF2091EF043091F004821BD3
:1019E000930B8838934108F061D9D091E804809135
:1019F0002001813021F48091A20587FD0DC086E091
:101A00002AEE31E090E0815058F491114FD9CD2B5E
:101A10008C2FDF91CF9108958EE122EF31E0F2CF4C
:101A2000F90141919F01411571F39F5FECCF962F12
:101A30002091A30522FF0EC0682F660F660F660F68
:101A4000692B6093EC045ED8AEDF9093EE04809334
:101A5000ED04089557C89091E804292F28232115F3
:101A600059F0809589238093E804811531F09BDF3C
:101A70008093EF049093F004089580E090E0F8CF15
:101A800092DF2091450430914604232B211521F04B
:101A900080938B0390938C032091470430914804EA
:101AA000232B211521F08093890390938A03E091E1
:101AB000C503F091C603309759F00680F781E02DF9
:101AC000309731F082E08093430483E494E00995F9
:101AD0000895611509F441C0E3E3E80FE33148F4E8
:101AE000F0E0EB55FA4C0C94DB3351DE819580939A
:101AF0004604C6CF4CDEFBCF4ADE81958093450479
:101B0000F8CF45DEFBCF63DE80934704F2CF5FDE84
:101B10008195FACF5CDE819580934804EACF57DE49
:101B2000FBCF815D990B21E030E001C0220F8A9547
:101B3000EAF780914404822B80934404DACF8091A9
:101B40004204816080934204D4CF80914204826039
:101B5000F9CF809142048460F5CF409145048D3CDB
:101B600059F48091460487FF0DC010924604411538
:101B700059F41092410408C08E3C81F480914604CF
:101B800018169CF3411581F0809147049091480408
:101B9000892B8111AECF10924004ABCF8F3C41F422
:101BA00047FFF0CF10924504809146048115E0CFA5
:101BB000803D19F41416B4F3E5CF90914704893DA4
:101BC00029F41916FCF610924704DCCF8A3D19F46B
:101BD00097FFD8CFF8CF909148048B3D29F497FF19
:101BE000D1CF10924804CECF8C3D19F41916CCF306
:101BF000C9CF9FE2980F983090F4815D990B21E056
:101C000030E0B90102C0660F771F8A95E2F7CB0179
:101C1000809590914404892380934404B3CF8D3DF3
:101C200031F4809142048E7F80934204ABCF8E3D8D
:101C300021F4809142048D7FF7CF8F3D09F0A2CF30
:101C4000809142048B7FF0CF2FB7F89460912802E7
:101C50007091290280912A0290912B022FBF089542
:101C6000FC019B0180911E0290911F02861797072D
:101C700040F0672B29F48091E8008E778093E8008C
:101C8000C90140E0009741F4411106C08091E8008D
:101C900082FF2FC080E0089520919E032115A9F1B5
:101CA0002530A9F12091E80023FD2DC02091E80006
:101CB00022FDECCF2091E80020FFE4CF3091F3002B
:101CC0002091F200009719F02830310558F041E0DA
:101CD0002830310509F040E02091E8002E7720936C
:101CE000E800D0CF41914093F10001972F5F3F4F23
:101CF000E9CF80919E03811541F0853041F08091BC
:101D0000E80083FFC3CF81E0089582E0089583E077
:101D100008958091180287FF13C08091E80082FF28
:101D200006C08091E8008B778093E8000895809149
:101D30009E038111F2CF089580919E038115D9F3FE
:101D40008091E80080FFF8CF8091E8008E77ECCF9B
:101D50002091E4003091E50095E6A9012091EC0086
:101D6000822F817020FF06C08091E80080FF06C0AE
:101D700080E008952091E80022FD1AC080919E0322
:101D8000811589F0853089F08091EB0085FD0FC0C9
:101D90002091E4003091E50042175307F9F29A953B
:101DA000E1F684E0089582E0089583E0089581E0FB
:101DB0000895E8EDF0E080818E7F80831092E2004C
:101DC0001092DA001092E100A0EEB0E08C918160F8
:101DD0008C9380818F77808319BCA7EDB0E08C91C4
:101DE0008E7F8C9380818F7E80831092170208955E
:101DF000E091C503F091C603309739F00284F38572
:101E0000E02D309711F060E209950895982F909396
:101E1000E900891771F07091EC002091ED0050916C
:101E2000F00021FD09C09F5F973089F78093E9009A
:101E30000895762F242F50E03091EB003E7F3093B1
:101E4000EB003091ED003D7F3093ED003091EB00E1
:101E500031603093EB007093EC002093ED005093D1
:101E6000F0002091EE0027FDDECF0895A0E0B0E065
:101E7000ECE3FFE00C94FE33C8EDD0E088818F7E68
:101E80008883E7EDF0E080818160808384E082BF19
:101E900081E08093170288818E7F888302EE10E0B4
:101EA000F80110821092DA0081EEC82ED12CF601D2
:101EB000108288818F778883888180688883888171
:101EC0008F7D888319BC10929E0310921602109287
:101ED00077031092150290EEE92EF12CF701808124
:101EE0008B7F808388818160888342E060E080E02E
:101EF0008DDFF60180818E7F8083F8018081816093
:101F00008083808188608083F70180818E7F8083D9
:101F1000888180618883CDB7DEB7E8E00C941A34FD
:101F2000E091D0039091CF0329E0E91302C080E053
:101F30000895AE2FB0E02E9FF0011124EF52FC4F18
:101F40003181361306C03081381303C03581341314
:101F500004C0FD013196E770E8CF81E0089535B106
:101F60003E7F25B121604FB7F89481E392E0FC01F8
:101F70000196508168E025B9000000C057FF35B9CF
:101F8000550F000000C000C000C035B900C06A9500
:101F900091F752E08538950751F74FBF8FE594E0F0
:101FA0000197F1F700C00000089581E08093E00000
:101FB00080E28093D8001092C9008FE19EE40197DF
:101FC000F1F700C0000087E090EBDC018093A405EE
:101FD0009093A505A093A605B093A70588E19CE082
:101FE0000FB6F894A895809360000FBE90936000A0
:101FF000FFCF0F931F93CF93DF938B01EA01909153
:102000009E03943051F58093E9008FEF9091E800A2
:1020100095FD06C095ED9A95F1F700008A95B1F708
:102020008091E80085FF19C093DE811111C0809175
:10203000E80085FD06C08091E8008E778093E80077
:10204000F3CFF80181918F018093F100219779F707
:102050008091E8008E778093E800DF91CF911F9107
:102060000F910895792F603229F440E250E0682FF3
:1020700082E0BFCF0895CF93DF93D82FC92F48E0D8
:1020800050E0682F792F81E0B4DF88E0ED2FFC2F3E
:10209000A0E2B2E001900D928A95E1F7DF91CF9135
:1020A0000895BC0140E250E084E0A3CFBC0146E0CB
:1020B00050E084E09ECFBC0143E050E084E099CF43
:1020C0009091A30592FB222720F9281779F080FB35
:1020D00092F99093A3056091A2057091A30584E005
:1020E00090E00E942B3582E00C942D0608951F93FA
:1020F000CF93DF93962F122F632F8430D8F495302F
:10210000C8F44F30B8F4C42FD0E0CC0FDD1F2EE15F
:10211000929FC00DD11D112496E9899FC00DD11D3C
:102120001124CE0189960E941135612FCE018A9625
:102130000E941135DF91CF911F9108958091200168
:10214000813061F58091A20587FF28C038DC80933B
:10215000F10140E250E065EA73E080EF91E00E9417
:10216000CC34892BD1F080E2E0EFF1E0A5EAB3E0D6
:1021700001900D928A95E1F7E091C503F091C603B5
:10218000309759F00480F581E02D309731F086E0EA
:102190008093F00180EF91E00995089510DC809321
:1021A000E80148E050E067EC73E088EE91E00E94BF
:1021B000CC34892B91F388E0E8EEF1E0A7ECB3E0B2
:1021C00001900D928A95E1F7E091C503F091C60365
:1021D000309719F30280F381E02D3097F1F288EE09
:1021E00091E0DACFCF93C82F8115A1F08238A1F406
:1021F00018DB81FD0FC089E373DBA0DF2FEF37EE23
:1022000083E0215030408040E1F700C0000089E3C6
:102210009BDB94DFCF910895833889F402DB80FD46
:10222000F9CF83E55DDB8ADF9FEF21EE34E091504B
:1022300020403040E1F700C0000083E5E9CF84385A
:1022400089F4EFDA82FDE6CF87E44ADB77DF8FEFB0
:1022500091EE24E0815090402040E1F700C0000062
:1022600087E4D6CF8CEF8C0F813A78F580912001EE
:10227000813069F0EAEEF1E080EF91E02191C21740
:1022800001F18E179F07D1F78C2F2ADBC2CF8091E7
:10229000A20587FFEFCFEC2FE695E695E695F0E0F7
:1022A000E051FE4F828190E04C2F477021E030E0FA
:1022B00002C0220F331F4A95E2F782239323892B12
:1022C00019F38C2F41DB3ADFDFCF80E28C0F8830AF
:1022D00048F4C77081E001C0880FCA95EAF70E94F0
:1022E000480697CF8BE58C0F833030F42C2F245287
:1022F000330BC901A5DA8ECFE8E5EC0FEB3148F4DA
:10230000F0E0EE0FFF1FE055FE4F80819181C0DAB3
:1023100081CF83E38C0F833108F07CCF61E08C2F79
:10232000D8DB78CF811509F445C0823849F479DAD1
:1023300081FF40C089E3D4DA01DF89E305DBFECE0B
:10234000833841F46EDA80FF35C083E5C9DAF6DE02
:1023500083E5F4CF843841F464DA82FF2BC087E44C
:10236000BFDAECDE87E4EACF9CEF980F913A30F3C6
:1023700090E2980F983050F4877091E001C0990F67
:102380008A95EAF7892F0E944E06D9CF9BE5980FD0
:10239000933018F480E090E053CA98E5980F9B3191
:1023A00018F480E090E074CA93E3980F933110F42E
:1023B00060E08FCB08951F93CF93DF93182FEB012D
:1023C00011DF209731F4812FADDFDF91CF911F9185
:1023D00008958FE99FE00197F1F700C00000219771
:1023E000F0CF811519F00E944806A8CE08958115F6
:1023F00019F00E944E06A2CE0895811531F09091F9
:10240000EB04892B8093EB0499CE0895811539F064
:1024100080959091EB0489238093EB048FCE0895EF
:1024200080915304811521F082E2F0DF1092530471
:1024300008951092E90480912001813011F5809176
:10244000A20587FF1EC0E2EFF1E08EE1DF011D92E1
:102450008A95E9F780E090E0F3D980E090E018DA1F
:102460001092EB046BDE86E0E3E4F4E0DF011D9202
:102470008A95E9F7109241041092400410924204A8
:10248000FFCAEAEEF1E086E0E1CFD3DF2FEF84E38D
:102490009CE0215080409040E1F700C0000088E1BE
:1024A0009CE00FB6F894A895809360000FBE9093BF
:1024B0006000FFCFAAE2B0E0E0E6F2E10C94033462
:1024C00088E192E0FC0101962091F100208322E056
:1024D00080329207B9F780911902893009F457C008
:1024E000C8F4823009F4B2C0833009F482C081306C
:1024F00081F18091E80083FFE6C0809118029091FD
:1025000019029A3008F0DFC0E92FF0E0E854FA4CE5
:102510000C94DB338A3009F489C08B3051F78091F9
:102520001802813231F780911C0290911D02892B93
:1025300001F78091E800877F8093E800EADB81E083
:1025400090911A02911101C080E08093200171DF07
:10255000D0CF80911802813A61F68091E800877FA0
:102560008093E80080911C0290911D02892B59F004
:1025700060E080E090E070E073DB8091E8008B77B2
:102580008093E800B6CF68E080E292E0F4CF8091DB
:102590001802813209F0ADCF80911C0290911D028A
:1025A0008D7F892B09F0A5CF8091E800877F8093EC
:1025B000E8008091E80082FF17C09091F3008091BD
:1025C000F200029731F48091F100813011F08630F1
:1025D00021F48091F10080931F018091E8008B77B6
:1025E0008093E80096DB85CF80919E038111E1CF37
:1025F00080CF80911802813A09F07BCF80911C0234
:1026000090911D02892B09F074CF8091E800877F9B
:102610008093E8008091E80080FFFCCF809120014A
:102620008093F1008091E8008E77DACF80911802D4
:10263000813209F05ECF8091E800877F8093E800C7
:1026400068DB80911B0280931E0153CF809118029A
:10265000813A09F04ECF8091E800877F8093E800AF
:102660008091E80080FFFCCF80911E01D9CF803897
:1026700089F0823841F580911C028F70873018F5FF
:102680008093E9008091EB0085FB882780F9109208
:10269000E90006C080917703880F90911502892B7D
:1026A0009091E800977F9093E8008093F10010925A
:1026B000F1008091E8008E7723C0811116C08091CF
:1026C0001A02813009F18091E80083FF0AC08091ED
:1026D000E800877F8093E8008091EB008062809320
:1026E000EB00AA96E3E00C941F34823061F78091EE
:1026F0001A02811581F01092E9008091E800877F2D
:102700008093E80006DBDFCF81E0933009F080E0C2
:1027100080937703F0CF80911C028F702FEF280FEA
:10272000263088F68093E9002091EB0020FFE3CF6C
:10273000933031F48091EB0080628093EB00DBCF2B
:102740009091EB0090619093EB0021E030E0A901C3
:1027500002C0440F551F8A95E2F74093EA00109299
:10276000EA008091EB008860E8CF8111ACCF109136
:102770001A021F778091E3008078812B8093E30019
:102780008091E800877F8093E800C3DA8091E800B9
:1027900080FFFCCF8091E30080688093E30083E0BA
:1027A000111101C082E080939E038DCF805882304A
:1027B00008F089CF80911A0290911B028C3D53E062
:1027C000950791F583E08A838AE289834FB7F8946D
:1027D000DE01139620E03EE051E2E32FF0E050935B
:1027E0005700849120FF03C082958F703F5F8F70E8
:1027F0008A30C0F0895C90E08D939D932F5F2431E7
:1028000061F74FBF8091E800877F8093E8006AE21C
:1028100070E0CE01019624DA8091E8008B778093F6
:10282000E80051CF805DE7CF292F332723303105D2
:1028300009F44EC078F52130310509F488C08BE5E4
:1028400090E0E8E7F2E02230310509F03CCF20913A
:10285000E800277F2093E80020911E0230911F029C
:102860008217930708F49C0140E02115310509F017
:1028700073C0411171C08091E80082FDCDCF80917D
:102880009E03811549F2853039F28091E80083FF7B
:10289000F2CFC2CF80911C0290911D0221323105EE
:1028A00009F446C02232310509F00DCF833091057D
:1028B00008F009CFFC01EE0FFF1FE15DFE4F019014
:1028C000F081E02D845D9E4FDC018C9190E010C082
:1028D0009C013327823021F12330310568F4232B0A
:1028E000B9F4E9E2F3E0E4918E2F90E0E9E2F3E05D
:1028F000009709F4E8CEABCF2330310509F0E3CEE1
:10290000E5EEF2E0E4918E2F90E0E5EEF2E0F0CF1C
:10291000EBE1F3E0E4918E2F90E0EBE1F3E0E8CF20
:10292000E3E0F3E0E4918E2F90E0E3E0F3E0E0CF2A
:102930008330910508F0C7CEFC01EE0FFF1FEB5C62
:10294000FE4F0190F081E02D89E090E080CF82E1A0
:1029500090E0E3EDF2E07BCF80919E03811509F4D6
:102960005BCF853009F458CF8091E80083FD54CFC8
:102970008091E80082FD7FCF8091E80080FF75CFD5
:102980009091F3008091F2002115310519F0883003
:10299000910550F041E0089709F040E08091E8008F
:1029A0008E778093E80061CF44914093F100319697
:1029B000215031090196E8CF803809F084CE80910A
:1029C000E800877F8093E800809116028093F100F1
:1029D00070CE811178CE10911A02123008F073CEA9
:1029E0008091E800877F8093E8001093160291D9C8
:1029F0001115D9F084E080939E0342E061EC81E000
:102A000005DA42E261EC84E001DA42E261EC82E064
:102A1000FDD942E260EC83E0F9D980919E038430D5
:102A200051F482E0809321014ECE8091E30087FD36
:102A3000E1CF81E0E0CF81E0F5CFCF93DF93EC01F0
:102A40004A855B856E857F850E940C0C9B819095E5
:102A50008091EB0489238093EB048C810E944E06C5
:102A60006DDB86E0FE0111928A95E9F7DF91CF9147
:102A70000895CF93DF93EC018D8181FD13C08260B7
:102A80008D838091EB049B81892B8093EB048C8157
:102A90000E94480653DB488559856E857F85CE01A7
:102AA0000E940C0C1092D8041092D7048D8180FDE6
:102AB00002C0CE01C2DFDF91CF9108950F931F9323
:102AC000CF93DF93843030F5653020F54F3010F52B
:102AD000C42FD0E0CC0FDD1F2EE1629FC00DD11DB1
:102AE000112436E9839FC00DD11D1124CE01899692
:102AF0000E94F034082F10E0102F0027CE018A9694
:102B00000E94F0349801282BC901DF91CF911F91C9
:102B10000F91089580E090E0F8CF462F672F209125
:102B2000A1033091A203232B81F4703F39F4403F7D
:102B300061F480919F039091A0030895753028F46B
:102B40004F3018F4843008F4B9CF80E090E0089555
:102B5000A0E0B0E0EEEAF5E10C94FF337C010091D7
:102B6000A1058091A005082BC3E0D0E010E0C801CA
:102B70000C2E02C0959587950A94E2F780FD09C056
:102B80002197A8F7D12C8D2DCDB7DEB7E7E00C94B7
:102B90001B34DC2EB7018C2FC0DF0E945407019735
:102BA00079F3F1CF0F931F93CF93FC018781908529
:102BB000009789F4858100811181811581F061156B
:102BC00071F0C801C5DFC82F682FC8010E949A059F
:102BD000B8018C2FA2DFCF911F910F910895C801EA
:102BE0000E94D005C82FF4CFCF93DF93D82FC92FE1
:102BF000AFDF6D2F7C2F91DF0E945407DF91CF91C3
:102C00000895FC0184818115B1F08781908500973A
:102C1000A1F00E945407282F92959F709630B9F02A
:102C200080F4925F9F70923030F4203FD1F058F4DE
:102C300081E0283E58F080E0089580819181D4DFC2
:102C4000EACF9A5FEFCF81E0243FA9F7089591E0A2
:102C5000813F09F090E081E0283E08F080E0892B78
:102C6000089581E00895382F292FCB01A32FB22F8B
:102C70008F3D9105A105B10520F48F5D9C4F0C940B
:102C8000F03480E0089585E290E00E94F0348731CE
:102C900089F486E290E00E94F034803159F487E2B2
:102CA00090E00E94F03491E08F3909F090E0892F94
:102CB0008170089580E0FCCFA0E0B0E0E2E6F6E1AC
:102CC0000C94FD33EC018881811509F1813009F004
:102CD00045C08981813051F48A81239660E570E096
:102CE000893311F060E070E066DBEDCF823021F4D3
:102CF0008A81239677DAE7CF833021F48A8123967D
:102D000011DBE1CF843041F022968111DCCFCDB7C9
:102D1000DEB7E9E00C9419348A81239620E030E094
:102D20009AE0682F6053770BAB016A30710560F051
:102D30002115310551F3EFE9FFE03197F1F700C0BC
:102D4000000021503109F4CF929FB001939F700D84
:102D500011249A01260F371F8991E3CFE82FF0E065
:102D6000E850FE4FB490282F26952695269530E002
:102D7000F901E851FE4FE4908770F12C082E02C053
:102D8000F594E7940A94E2F7E0FAEE24FF24E0F8E1
:102D9000F901E852FE4FC490D12C082E02C0D59400
:102DA000C7940A94E2F7C0FACC24DD24C0F8F901F4
:102DB000E853FE4F049110E002C0159507958A95DF
:102DC000E2F701701127E114F10411F081EE0ADA43
:102DD000C114D10411F086EE05DA60E070E08B2DAD
:102DE000EADAC114D10411F086EE9CDAE114F104A0
:102DF00011F081EE97DA0115110521F060E070E025
:102E00008CE2D9DA21965FCFAAE0B0E0EAE0F7E100
:102E10000C94F933C0909C03D0909D0381E090E026
:102E200090939D0380939C03812C912CE12C540161
:102E3000F12C14C0F80125913591472D6F2D8E2D61
:102E400056D90E5F1F4F73948FE07812F3CF9FE037
:102E5000A90EB11CF394E5E0FE1639F08501000FD0
:102E6000111F035D1C4F712CE5CFE394FBE48F0E23
:102E7000911C84E0E812DBCF1A8219821C821B822B
:102E80001E821D8218861F8288EC90E09A878987AF
:102E900001E812E0FE0131967F014AE050E0B801FE
:102EA000C7010E942F35065F1F4F5701013DF2E019
:102EB0001F0799F78AE0F70111928A95E9F74AE02E
:102EC00050E0B801C5010E942F35065F1F4F013247
:102ED000F3E01F07A1F7D0929D03C0929C032A96AE
:102EE000EDE00C941534AAE0B0E0E9E7F7E10C94CA
:102EF000FE33E5E8F2E080E5DF011D928A95E9F70F
:102F0000E1EFF4E088E3DF011D928A95E9F785E8B7
:102F1000C82E82E0D82E7F0101ED12E0F701D182A8
:102F2000C0824AE050E0B801CE0101960E94E03430
:102F300088E0FE013196D60101900D928A95E1F765
:102F400089859A85D70113969C938E931297BAE040
:102F5000CB0ED11CE7E0EE0EF11C065F1F4F0132D5
:102F6000F3E01F07D9F62A96E8E00C941A34282FCC
:102F7000CB01283070F44AE0249F90011124B9015C
:102F80006F577D4F4AE050E00E94E03480E090E0CF
:102F900008958FEF9FEF0895AAE0B0E0E2EDF7E12A
:102FA0000C9404349C0197558115914068F4BE013E
:102FB0006F5F7F4F822FDBDF892B31F489859A8504
:102FC0002A96E2E00C94203488EC90E0F9CFA0E05F
:102FD000B0E0EDEEF7E10C94FF33162FD72FC42F9E
:102FE000D22E8115A1F04093DB040E94D30C909364
:102FF000140280931302C77081E001C0880FCA9544
:10300000EAF7EFD9CDB7DEB7E7E00C941B34909127
:10301000DB04491335C0E0901302F09014020E94C3
:10302000D30C9C012E193F097901812F9D2FB4DF0C
:10303000E816F90628F5D0E2DD0DCD1591F0C77040
:1030400011E0812F01C0880FCA95EAF7D0D9D83096
:1030500040F48D2D877001C0110F8A95EAF7812FFA
:10306000C0D960E070E0802FA6D9D83058F62D2D59
:10307000277081E001C0880F2A95EAF7B8D9C2CF3E
:10308000C77081E001C0880FCA95EAF7F7CFA0E0CA
:10309000B0E0EDE4F8E10C94F833FC018280648048
:1030A00081E08483E5E8F5E09490E4E0F6E0E491E3
:1030B0000091E2040695015810E0000F111F012F46
:1030C0001127CDEDD2E0C12CD12CAA24AA94B12C89
:1030D00077247A94E919EE2EF12C83E0881630F4E7
:1030E0008091E00488838091E104898361101AC093
:1030F0001B821A824A81493C08F048EC960169819A
:1031000088810E94F3088FEFC81AD80A25968CE1AF
:10311000C816D10411F70E941609CDB7DEB7EEE04C
:103120000C9414348B818115E9F081508B83789E47
:10313000C00111246C8170E00E94B433FB01FF27B1
:10314000EB57FA4F8491E82FE9197E9EC0011124B4
:10315000B7010E94B4338091E204689FB00111244A
:103160007A83C8CF0E94A834B5010E94C833801763
:1031700091070CF0BFCF83E0881688F00E94A83436
:10318000B5010E94C83388830E94A8342091E104CD
:103190002695622F70E00E94C833280F29831A8277
:1031A0008091E204893C20F088EC8C838B83A2CF51
:1031B0008431D8F784E1F9CF0F93CF93DF93CFED2C
:1031C000D4E0488159816A817B8188E090E00E9447
:1031D0002335288139814A815B816C817D818E8193
:1031E0009F8100E20E944634622F83E290E00E94B9
:1031F0001135DF91CF910F910895EFEDF4E085E067
:10320000808311828FEF828388EC83831482CF01C5
:10321000D3CF8091E304833018F48F5F8093E3046D
:103220008FED94E0C9CF8091E304811519F08150AE
:103230008093E3048FED94E0BFCFA0E0B0E0E3E241
:10324000F9E10C94F933082FF62E142FE22E909109
:10325000DF0490FF26C0E92FE695E695AE2FB0E09B
:10326000A55CBE4F8C918093DD049C7F9430F1F47B
:10327000842F493C08F088EC602F7F2D0E946C0859
:10328000962F672F482F892F0E942B090093E00467
:10329000F092E1041093E204E11419F08FED94E050
:1032A0008BDFCDB7DEB7EDE00C941534823019F426
:1032B0001091E204EBCF863019F40091E004E6CFE0
:1032C0008930D9F3893111F7E9518E2F8170782E29
:1032D000E695F0E0EB57F94FE491CE2FD0E0A12C2A
:1032E000B12CC12CD12C8CE1882E912CC501B401BC
:1032F0000E94B433802F711015C0860F412F193CE6
:1033000008F048EC96016F2D0E94F3088FEFC81A61
:10331000D80AAC0EBD1E8CE1C816D10439F70E9444
:103320001609B4CF861BEACFEFEDF4E0818121E0EE
:1033300043816281885F81CFEFEDF4E0818121E0FC
:1033400043816281885079CFEFEDF4E0628121E121
:10335000620F08F46FEF21E0438181816ECFEFEDC2
:10336000F4E0628121E1621B08F460E021E0438126
:10337000818163CFEFEDF4E0438121E1420F08F456
:103380004FEF21E06281818158CFEFEDF4E043817E
:1033900021E1421B08F440E021E0628181814DCFB0
:1033A0009091DF0490FF2CC0811559F18B3258F5B4
:1033B0008F73880F880F9091DF049370892B80930F
:1033C000DF04611519F08FED94E0F6DE6091DF0403
:1033D0006695669570E04BE050E087E091E00E94D2
:1033E000BF34892B91F01092DE0481E08093860334
:1033F00020E04091E2046091E1048091E0041DCF5F
:10340000089581E0D6CF8AE2D4CF81E08093DE04B4
:103410000E94D30C9093840380938303E6CF809122
:10342000DF04869586958F5F8B3208F081E061E03E
:10343000B7CF8091DF04869586958A9509F48AE254
:1034400061E0AECFA8E0B0E0E8E2FAE10C94F63338
:103450007C01DC0114968C91811509F4BDC161E0F9
:10346000C701A0DB8C01F7018581811521F18091D5
:10347000D7049091D8040097F1F008171907D9F0F4
:10348000FC01FF27887F9927892B09F072C0A4E0EF
:10349000EE0FFF1FAA95E1F7E95AFB4F8581846083
:1034A000858311830083CF01E4DA1092EB0461E09D
:1034B000C70178DB8C01D70115968C91811509F431
:1034C000E3C0C80197578038910508F06BC10031FF
:1034D00008F072C16EED70E080E090E0C4DB811115
:1034E0006BC1812C912C5401011146C004E09E0156
:1034F0002F5F3F4F6901D601E02F1D92EA95E9F752
:1035000024013501FFEF4F1A5F0A6F0A7F0AC501D8
:10351000B401A9DB8983811509F44EC1813009F01A
:10352000B0C0A50194012E5F3F4F4F4F5F4F2D83D9
:103530003E834F835887C301B20195DB182F8A83DE
:10354000811509F439C18FEF810F833078F56D81D2
:103550007E818F81988587DB8B83811511F0C60171
:10356000ABDB2401350133E0430E511C611C711C9F
:103570001AC0E0E0F0E092CFBFED8B169104A104F9
:10358000B10409F419C1C501B4016DDBEFEF8E1A66
:103590009E0AAE0ABE0A8111EFCF0150A5CF4D8021
:1035A0005E806F80788453014201A5CF8BEF810F3D
:1035B000833090F52401350143E0440E511C611C19
:1035C000711C6D817E818F8198854DDB8B83811588
:1035D00051F3C301B20147DB8C83811108C0240180
:1035E000350154E0450E511C611C711CDCCF8B81F0
:1035F0009C818130AFEF9A0710F0982F8827163002
:1036000029F0173031F00E942D28E9CF0E94C927F8
:10361000E6CF0E94FB27E3CF143009F0C0CF6D81C5
:103620007E818F8198851FDB182F24013501B4E03E
:103630004B0E511C611C711CC501B4016D5F7F4FA5
:103640008F4F9F4F10DB111509F4B6C0811509F497
:10365000B3C08150990B4FEF489F9001499F300DA7
:103660001124E12FE150FF0B2E0F3F1F2150310994
:1036700008F499CF8FE99FE00197F1F700C00000AF
:10368000F5CFC60119DB8FCF0115A7E51A0708F49E
:10369000B7C00115B8E51B0708F0A9C66801E7E542
:1036A000DE1A69E474E08C2D62DC892B31F5C601E9
:1036B00074E0880F991F7A95E1F7FC01E95AFB4FF6
:1036C0002281213009F05AC02091490430914A04E6
:1036D000232B99F020914B0430914C04232B69F05B
:1036E00020914D0430914E0440914F04509150046C
:1036F000242B352B232B09F44BC0809153048115C7
:1037000009F467C1C090E904D090E8040E94D30C8A
:1037100088579C4E9093550480935404F7018581FB
:10372000811509F456C18D2D8C298D79811122C105
:103730000115F0E51F0708F0BAC0011520E41207D3
:1037400008F030C1063E110509F4DFC0C8019052EF
:103750008115904208F02DC1D70116968C918031C9
:1037600008F400C1C80199271092EB048D3291052D
:1037700009F0B6C082E08093EB041FC1223009F04B
:10378000BCCF20914D0430914E04232B09F4B5CFCA
:10379000FC01E45AFB4F20812E7F2083895A9B4FE6
:1037A00068D9ABCF0337FCE71F0751F5809153046D
:1037B0008115B1F00E9410128091EC048770811580
:1037C00059F0F7018581811539F08091A30582FFB9
:1037D00003C082E00E942D062896E0E10C9412348A
:1037E0001092E9040E9456060E94D30C88579C4E02
:1037F000909355048093540481E080935304DCCF6C
:10380000023A22E51207C1F158F4C801905281151D
:10381000904218F1013E110579F1053E110503C0F2
:10382000023B52E5150709F068CF25EE30E027701E
:10383000332781E090E001C0880F2A95EAF72091B4
:103840005604309153043115F9F0F70135813115E3
:10385000B1F0282B20935604AFCFD70116968C9148
:10386000803108F04ACF812F99278F7199278230B4
:10387000910511F04297D7CF21EE30E0D8CF809557
:1038800082238093560498CF322F3823311509F4C0
:1038900034CF982F90959223909356040E944E0611
:1038A000D70115968C91811509F486CF26CF003E5D
:1038B000B2E51B0708F049C0003CE2E51E0728F509
:1038C000003AF2E51F07E8F4003622E51207E8F4B3
:1038D000C801925580349105C0F01092EB04C801E4
:1038E0008E32910508F0BCC08832910508F063C0A3
:1038F0008E31910508F061C004974A9708F43ACFD9
:1039000039C0043B32E5130741F7F7019581911562
:1039100009F488C51092DB04980130572332310531
:1039200008F069C584E090E00E94FD349093A305FF
:103930008093A205F801E150F047E232F10508F06A
:10394000E3C0EE53FA4C0C94DB3309374CE7140711
:1039500028F407375CE71507C0F6BFCF0B378CE7B5
:103960001807D2CF812F8F71843179F2863149F4D3
:103970001092EB040E941012809156040E94480697
:1039800028C00E941012809156040E944806F80137
:10399000E851FC47E730F10508F0B7CFEC51FA4C9D
:1039A0000C94DB33D70116968C91803108F0DACE77
:1039B000EECFC801D9CE8A97E9F6809156048115D9
:1039C00031F08091EB0492E089278093EB040E9410
:1039D0009E10C801975581159140C8F65801F8EF1F
:1039E000AF22BB24A114B10409F0E6CEF801FF27F1
:1039F00054E0EE0FFF1F5A95E1F79F01295A3B4F04
:103A00006901D70115968C91E45AFB4F908180FB98
:103A100090F99083811559F10E94D30C9093DA04A8
:103A20008093D904F60182818F5F82838091EB04B9
:103A30009091E904892B83838091E80484834681F3
:103A4000578166857785C6010E940C0CD6011596B4
:103A50008C9181FF5801B092D804A092D70455CF21
:103A60008C34910509F4A9CF8D329240A5CFF9018C
:103A70004485558566857785C9010E940C0CD60161
:103A800015968C9181FF41CFC6010E941D15809132
:103A9000D7049091D8040817190709F036CF10926F
:103AA000D8041092D70431CF06E221EE41EE6AE14C
:103AB0007CE7F701858108C007E225EE45EE6BE162
:103AC0007CE7D70115968C9182DA76CE06E221EE5C
:103AD00040EE68E17CE7EDCF07E225EE44EE69E1D8
:103AE0007CE7EFCF06E221EE42EE6CE17CE7E1CF2E
:103AF00007E225EE46EE6DE17CE7E3CF08E221E048
:103B000045EE6EE17CE7D5CF8091A2058160809380
:103B1000A2056091A2057091A30584E090E00E9447
:103B20002B350E94191248CE8091A305886080939E
:103B3000A305EFCF8091A2058260E9CF8091A20515
:103B40008460E5CF8091A2058860E1CF8091A305D4
:103B50008160EDCF8091A3058260E9CF8091A205BD
:103B60008061D5CF8091A2058062D1CF8091A205DE
:103B70008064CDCF0E9419128091A2058068C7CFC2
:103B80008091A2058C60C3CF8091A3058360CFCFC5
:103B90008091A2058E7FBBCF8091A305877FC7CF81
:103BA0008091A2058D7FB3CF8091A2058B7FAFCF8F
:103BB0008091A205877FABCF8091A3058E7FB7CF81
:103BC0008091A3058D7FB3CF8091A2058F7E9FCF7B
:103BD0008091A2058F7D9BCF8091A2058F7B97CF8F
:103BE0000E9419128091A2058F7791CF8091A20532
:103BF000837F8DCF8091A3058C7F99CF8091A20583
:103C0000992782FF939590FB82F990FB83F97FCFF0
:103C10008091A305982F909590FB80F990FB81F9F6
:103C200086CF9091A205892F8F7B96FF80646FCFFE
:103C30000E9419129091A205892F97FB87F980584D
:103C400066CF61E08EE090E00E94113562CF60E0C7
:103C5000F9CF9091A205892F8F7E94FF806157CF75
:103C60009091A205892F8E7F90FF816050CF909117
:103C7000A305892F877F93FF886059CF89E2CDC341
:103C800089E2DBC38272F801E052F847EB30F105BC
:103C900008F04CC0E551FA4C0C94DB330737FCE7D5
:103CA0001F0709F047C081E00E948C0565C0809124
:103CB000DF0480FF0BC08E7F8093DF048FED94E0E4
:103CC0007BDA1092DE040E94160976CD8160809323
:103CD000DF0461E08695869563DB6ECD811521F06A
:103CE000A8DB6ACD8115E1F39ADB66CD811521F061
:103CF00023DB62CD8115E1F317DB5ECD811521F069
:103D00002EDB5ACD8115E1F31FDB56CD811521F055
:103D10003CDB52CD8115E1F32DDB4ECD811521F039
:103D200082DA4ACD8115E1F374DA46CD07372CE704
:103D30001207F9F008373CE7130721F19801205EDC
:103D400032452032310518F5911121C00F7181E003
:103D500090E0AC0102C0440F551F0A95E2F78A01BA
:103D6000642F83E090E00E941135802F0E947C0533
:103D700023CD81E00E94820543E062E081E00E9461
:103D800004061ACD82E0911509F48ECFF3CF40914D
:103D9000E7048091A105282F30E02095309570E050
:103DA00024233723232B19F048234093E7040B37B0
:103DB0005CE7150741F4911509F4FECC0E946905F2
:103DC0000E94920BF9CC003482E5180708F055C028
:103DD0000032A2E51A0708F057C00115B0E51B072D
:103DE00050F50115E0E41E0708F064C0911509F4D0
:103DF0007AC00A35BCE71B0709F4D2C008F0B7C087
:103E00000130FCE71F0709F4C9C003302CE7120793
:103E100009F4BEC001151C4709F065C00E941912C3
:103E20008FEF94E3ACE081509040A040E1F700C0F8
:103E300000000E94D50F9801305521153240B0F690
:103E4000980145E0369527954A95E1F7822F8F70C6
:103E50002091E70430E041E050E0082E02C0440F1A
:103E6000551F0A94E2F724233523232B09F4BECFF0
:103E70009111A6CF1092E904D2C29801205C32457C
:103E80002032310508F0B2CF802F8F712091E704E6
:103E900030E041E050E0082E02C0440F551F0A9464
:103EA000E2F724233523232B09F4A0CF911509F43D
:103EB00083CC86CFD70116968C91803108F096CFAF
:103EC000911111C0212F2F7081E090E002C0880F66
:103ED000991F2A95E2F72091E70430E0822393238B
:103EE000892B09F069CCD70117968D919C91009789
:103EF00009F45AC00E9454078C01D7011596BC9052
:103F000015971696AC90A2942FE0A2228091EC0413
:103F10008770811501F1CB2CB114F1F0812F807FD6
:103F2000803461F080E2800F8830A8F0812F807E9D
:103F3000803221F4023078F0A11469F08091A30559
:103F400082FF09C082E00E942D068091EC048770F8
:103F5000CC24C3948111C12CE12FE295EF70103C69
:103F600008F095C0F0E0EA50FA4C0C94DB330B35C6
:103F70004CE71407B9F08091A305002482FF039455
:103F8000802D0C351C4709F0AECF0E946010ABCFDE
:103F90006FEF7FEF80E090E00E942B350E9445128A
:103FA00081E0F3CF80E0F1CFF7018581C080D1803F
:103FB000811569F0C6010E94A815182F682FC60147
:103FC0000E949A05B601812F0E948D1593CFC601DC
:103FD0000E94D005182FF6CFB12FBF70DB2E103105
:103FE00018F0D29490EFD922B114A9F0D11459F05D
:103FF00080E2800F883010F0011107C08D2D0E94E3
:1040000048060E949E10802F40C08091EB048D29AD
:104010008093EB04F6CF802F0E949211D114B9F156
:1040200080E2800F883010F0011104C08D2D0E94B5
:104030004E0606C0D0948091EB048D218093EB0452
:104040000E949E1024C0E12FEF70DE2E107F1032F0
:1040500019F0D29480EFD822011549F0013009F40B
:1040600082C0B11409F48EC0A114A1F1CCCF80910B
:10407000A30582FD2BC0B11419F1D11429F08D2DA7
:104080000E9448060E949E1080E00E94F210C11417
:1040900009F4D8C08091EC0480FDD4C0D7011596F6
:1040A0001C928695869586950E948205C701CAD97D
:1040B0008091EC048695869586950E948C05C2C0F9
:1040C00080E00E949211D11411F3B0CFB11469F1C4
:1040D000A11004C08D2D0E94F111D9CFF1E0AF12D3
:1040E00010C01091E8048D2D8123D81681F20E9412
:1040F000D30C9093F0048093EF041D291093E804EF
:10410000C6CF25E0A212C3CF8D2D0E94F1118D2DB7
:104110000E942B0D8091EA049D2D9823D91609F455
:10412000B6CF8D298093EA04B2CFA11012C08D2D95
:104130000E94F7118D2D0E942B0D8091EA049D2D78
:104140009823911509F4A3CFD094D822D092EA04F1
:104150009ECF31E0A3129BCF8091E9048D21811580
:1041600009F495CFE4CFB11429F046E0A41608F085
:104170008ECFB0CF55E0A51608F089CF8D2D0E94C7
:10418000F71185CFA114D1F3093349F48FEF97EEDE
:10419000A3E081509040A040E1F700C00000802FD4
:1041A0000E94921174CF812F869586958370811518
:1041B00061F0813009F06BCFC8019370B11002C07B
:1041C00080E090E00E94480C62CFC8019370B1106B
:1041D00002C080E090E00E94200C59CF6B2D802F10
:1041E0000E94690D54CF812F8370811138C0B110A6
:1041F00027C0402F429546954770440F440F802FAB
:104200008F70042E01C0880F0A94EAF7202F2071C6
:1042100004FF07C02FE030E001C0220F4A95EAF703
:1042200020951695169513701230A1F0133081F079
:104230003091A005113059F0822B83230E947C0518
:104240000E94110C60E0C7010E94D215C5CA832BE1
:10425000822BF4CF822B9091A0058927EFCFB11448
:1042600051F110FFEDCF402F429546954770440F16
:10427000440F802F8F70042E01C0880F0A94EAF734
:10428000202F207104FF07C02FE030E001C0220F73
:104290004A95EAF72095169516951370123089F015
:1042A000133069F03091A105113041F0822B832346
:1042B0000E947F05C5CF823018F2D5CF832B822B89
:1042C000F7CF822B9091A1058927F2CF1F70B114EF
:1042D00039F0812F0E948205802F0E94F111B0CF0A
:1042E000802F0E94F711812F0E948C05A9CF023FD9
:1042F00071F170F4003FC9F0013F91F0B11409F47D
:1043000065C0A11409F45FC0802F0E94F21098CFFD
:10431000033F21F1043F91F78091A30582FD2AC05C
:10432000812F8F71B11401F316C0B11469F0B5E09B
:10433000AB1608F085CF1F7181E090E0012E01C01F
:10434000880F0A94EAF7BECFE6E0AE16F2CF812FCF
:104350008F71B110C9CF0E94820572CF80E0B11475
:1043600009F4A6CF1F7181E0012E01C0880F0A94C5
:10437000EAF79ECFB114C1F08091EC0487708430CD
:1043800049F41092EC041092EE041092ED04812F87
:104390008F71AACFF5E063E0AF1608F051CF812FFF
:1043A0008F710E94170D4CCF25E0A21640F010929D
:1043B000EC041092EE041092ED0464E0F0CF81E082
:1043C0000E942D063DCF812F8F71C5CFA114F9F228
:1043D000093349F43FEF47EE53E03150404050403D
:1043E000E1F700C00000802F0E94921129CF03370F
:1043F000FCE71F0759CA8091E90406312CE7120730
:1044000009F040CC8A7A91E0811101C090E090934C
:10441000DC04811509F432CC85E30E94700C0E9403
:104420009E10CAC906313CE7130709F037CC8091CA
:10443000DC04811509F424CC85E30E94A40CEFCFA1
:10444000A0E0B0E0E6E2F2E20C94FF3380911F04BA
:10445000803108F049C080911E04811509F444C0E0
:10446000C091D00389E0D82E8091CF038C17E1F161
:10447000EC2EF12CDC9EE0011124FE01EF52FC4FEA
:1044800084818115B1F1918180911A04981331C012
:1044900090818091190498132CC08581811129C0C5
:1044A0000281138180911B0490911C04081B190B3D
:1044B00060E089E194E00E94D2150E94CC170817B1
:1044C0001907B8F480911F048F70806180931F04D6
:1044D000C952DC4F88818F708061888389E194E0C4
:1044E0000E94221A0E942306CDB7DEB7E7E00C94A3
:1044F0001B34E7012196C770B7CFAFE0B0E0E3E827
:10450000F2E20C94F7338C0186E0F801DE011A9692
:1045100001900D928A95E1F7F801F580E48089E138
:10452000882E84E0982E80911D04811117C0E1141B
:1045300091F0F11409F480C1C8010E94011681159F
:1045400009F47AC189E0F801A9E1B4E001900D9283
:104550008A95E1F775DFFF24F3946AC0A280B380E7
:10456000D0901E0480911B0490911C043501681AA0
:10457000790AD11409F411C1C080518060E089E149
:1045800094E00E94D2150E94CC176816790608F0B4
:10459000B6C0E11401F380911A04F8019181E09012
:1045A0001F04F0E1EF1608F064C0981320C090914A
:1045B0001904F801808198131AC0209120043091C9
:1045C0002104878190852817390789F4F1104BC0A1
:1045D0008E2D8F70806180931F0489E194E00E948A
:1045E000221A80911F04F8018683F12C21C0F1105A
:1045F0003AC040E0652D8C2D0E94900F40E0652D63
:104600008C2D0E94900FF82E8111EFCF8A859B850B
:104610000E94F415292F22952F70903470F49F700A
:104620002230A0F09115B1F0F8019681903190F40C
:104630008F2D2F96EFE00C9413342A5F2F702230C9
:1046400068F0C8010E94221AFD2CF2CF911511F0DA
:10465000811571F3805E883058F3F3CF803F40F3CB
:10466000815F8330F9CF80911F04816080931F04A4
:10467000BCCF98131EC090911904F8018081981343
:1046800018C020912004309121048781908528173B
:10469000390779F4F1100DC0E682C8010E94221A90
:1046A00089E0F801A9E1B4E001900D928A95E1F763
:1046B00052CFC8010E940116811509F4BDC0F11442
:1046C00009F4BAC080911F04803208F43BCF809176
:1046D000190490911A049A838983BC82AB828091D9
:1046E0001D048D831E82EF8280912004909121040D
:1046F00099878887CE0101960E94221A23CFD090F5
:104700001F04F0E1DF1650F489E194E00E94221AC0
:1047100089E0F40111928A95E9F767CFE11409F471
:104720001ACF90911A04F801818198131AC09091C0
:1047300019048081981315C0209120043091210420
:10474000878190852817390761F4F1100AC0D68255
:10475000C8010E94221A89E0F40111928A95E9F7B2
:10476000FACEC8010E940116811509F465C0F11442
:1047700009F462C080911F04803208F4E3CE809176
:10478000190490911A049A838983BC82AB82809128
:104790001D048D831E82DF82A7CF60E089E194E053
:1047A0000E94D2150E94CC176816790608F0B0CF87
:1047B000E11409F4D0CEF11409F43EC090911A042A
:1047C000F801818198132EC090911904808198136B
:1047D00029C02091200430912104878190852817D9
:1047E000390701F580911B0490911C04A81AB90A9D
:1047F000F8ECAF16B10408F053CF80911F0480FD90
:104800004FCF803108F44CCFF8018683982F907FEA
:10481000903F09F442CF982F907F905F8F70892B43
:1048200086833BCFC8010E94011681118BCE8091F7
:104830001F04816080931F04C8010E94221A8BCE3E
:10484000A2E1B0E0E6E2F4E20C9402340A871B87AE
:104850002C873D874E875F87688B798B8A8BCE014B
:104860000A964BDE811128C02091CF033091D003EE
:1048700089E0FE013A96DE01119601900D928A952B
:10488000E1F78E858115C1F0822F90E00196877047
:10489000992738171906D9F099E0929FD001112471
:1048A000AF52BC4FFE01319601900D929A95E1F7FF
:1048B0008093CF030E94230619E08091D00390914A
:1048C000CF03891312C06296E4E00C941E340E9458
:1048D00019121092CF031092D00389E0E9E1F4E0BD
:1048E000DF011D928A95E9F7E7CF189FC0011124D7
:1048F0008F529C4F02DE811531F38091D00390E0FE
:104900000196877099278093D003D7CFEF92FF92BB
:104910000F931F93CF93DF9380919D05E091300219
:10492000CDE0811130C0CDB7DEB7E6E00C941C3489
:10493000D1E0DE0FD0933002EE2EF12CCE9FF001AD
:104940001124EB5CFA4F84818115E1F08781908519
:10495000892B21F481859285019651F40081118182
:10496000228133814481558166817781808568DF2A
:10497000CE9DF001CF9DF00D1124EB5CFA4F148217
:104980001092EB04ED2F80919D05E81788F21092AC
:104990009D0510923002C7CFA4E0B0E0E2EDF4E252
:1049A0000C94F53320913405298397E0992E01E08A
:1049B00010E02DE0322E34E0532E88248394809131
:1049C00033059981891307C0A1DF0E94550B2496F6
:1049D000E1E10C9411349981892F90E09C838B83C1
:1049E000FC01EE0FFF1FE75DFA4F80819181989ED9
:1049F000D001999EB00D1124FD01EF50FB4FFA83B9
:104A0000E983248121115BC060909D05E5E3F5E019
:104A100060E070E0712C661508F04FC0A384B48488
:104A2000A981BA81CD90DC902FEF3FEF412C442D2E
:104A300050E07601E40CF11CE40CF11CD701ED9080
:104A4000FC90E114F10439F0AE14BF0409F0A9019F
:104A500043949A01ECCF2F3F3207D1F1D80102C025
:104A6000AA0FBB1F2A95E2F77A2A9801042C02C0EC
:104A7000220F331F0A94E2F7A9014150510974161D
:104A8000150629F5369EF001379EF00D1124EB5CDA
:104A9000FA4F989ED001999EB00D1124AF50BB4F94
:104AA00012962D913C911397308727835482108260
:104AB00011829287818715968C920E94660B8B815A
:104AC0009C8101969A8389838370898378CF14822D
:104AD0006F5F7F4F3D969FCF10929F0510929E056E
:104AE0001092220180913305809334050E94550B6A
:104AF0000DCFACE1B0E0EFE7F5E20C94F4334B8B73
:104B00005C8B6D8B7E8B8F8BB92E988FA92E91111C
:104B10001092EB04188A198A1A8A86E0FE017396AD
:104B2000DE011A9601900D928A95E1F75F888091D7
:104B3000A30582FF1FC00E94D30C2091ED04309189
:104B4000EE04821B930B8838934138F08091EC047B
:104B500082FD03C082E00E942D060E94D30C2091AA
:104B6000EF043091F004821B930B8838934110F0CE
:104B70000E9456065114D9F05E86BF8661E0CE01D0
:104B80000A960E94D21561E0CE010A960E94D215C3
:104B900061E0CE010A960E94D2154C0180356CE787
:104BA000960791F4A11419F181E0809322015E86A9
:104BB000BF860A851B852C853D85452D5B2D688923
:104BC00079898A893DDECDC081359C4721F4A114C5
:104BD00071F082DFECCF82E588168CE7980639F415
:104BE000A11429F0809122018111F3CFDDCF41EF93
:104BF000E42E44E0F42E412C612C712CD7016D91F0
:104C00007C91CC24CA94DD24DA9480E0282F30E013
:104C1000FB01E80FF11DE80FF11D408151814115A5
:104C2000510539F08416950609F096018F5F6901E8
:104C3000EDCF10E0BFEFCB16DB0609F44EC0F70155
:104C4000448110912201411110E0D70115963C904A
:104C5000159716969C911697A11409F405C1111584
:104C600009F402C1311017C021E030E00C2C01C062
:104C7000220F0A94EAF7922B16969C932091310505
:104C8000309132052233310530F422E330E03093A5
:104C9000320520933105E1E0F0E002C0EE0FFF1F86
:104CA0008A95E2F7CF010197D70116962C91281724
:104CB000190699F4C0909E05D0909F05C114D104A7
:104CC00009F453C00E94D30C8C199D09C39708F4B2
:104CD0004CC081E0F701848311E0412ABFEF6B1AD9
:104CE0007B0AE7E0EE0EF11CF8E06F16710409F0A4
:104CF00085CFA11409F417C1411409F414C10E940D
:104D0000D30C90939F0580939E0580919D058830DC
:104D100040F591E0980F90939D0599E0FE013A9639
:104D2000DE01119601900D929A95E1F75D82BE82A7
:104D30002DE0829FC00111248B5C9A4F29E0FE0177
:104D40003196DC0101900D922A95E1F72FEF3FEFAC
:104D5000DC011A963C932E9319971C969C928E9286
:104D60001B976C96E2E10C941034209134058091ED
:104D70003305922FE0E0F0E001E0281709F448C085
:104D8000422F50E0FA01EE0FFF1FE75DFA4F20803F
:104D9000318037E0329DF001339DF00D1124EF504A
:104DA000FB4F608171817C8F6B8FB0E030E0A0E0C1
:104DB000EB8DFC8DEA0FF11DEA0FF11DC080D18053
:104DC000C114D104E1F0F7010190F081E02DFA8FD8
:104DD000E98F30E007C0E1E0C616D70609F0E0E051
:104DE000BE2B3F5FE98DFA8DE30FF11DE30FF11D3F
:104DF000608171816115710571F7AF5FD9CFB11510
:104E000081F13A17C8F4E1E0D7011496EC93F70169
:104E100090933405EE15FF0509F45FCF90E0FC0197
:104E2000EE0FFF1FE75DFA4F71826082019683707B
:104E300099278093330551CF37E0329DF001339DA0
:104E4000F00D1124EF50FB4F0483EE15FF05F9F22E
:104E5000291302C09F5F93709A012F5F3F4F237009
:104E60008CCFE0E0F0E0F8CF292F30E0311024C003
:104E700061E070E002C0660F771F8A95E2F7CB0110
:104E800001972817390791F010E0E1E0F0E002C047
:104E9000EE0FFF1FCA94E2F76F01C094D701169678
:104EA0008C9116978C2116968C9317CF411569F328
:104EB000C3010E94660BE8CFA9010C2C02C05595D6
:104EC00047950A94E2F7C901019782239323892B1E
:104ED00039F540FF25C0D70112968D919C91892B01
:104EE000D1F087E0FE013196DF011D928A95E9F746
:104EF0000E94D30C9C018B839C8384E08D83F701FB
:104F000092818381792F9887898709811A8144E06A
:104F10005E816F8195DCD70115961C92132DB5CF5C
:104F2000142F1170B2CF90913405809133059817EA
:104F300031F032DDB1E04B1609F413CF38CEE6DCA8
:104F400010929F0510929E050E94550BF3CFA6E08C
:104F5000B0E0EDEAF7E20C9402340E94D30C8C012D
:104F60008091A3039091A4038017910771F0198297
:104F70001A820E94D30CBC0149815A8180E090E0E2
:104F8000B8DD1093A4030093A3032696E4E00C94E9
:104F90001E34A6E0B0E0EFECF7E20C9402348C0192
:104FA0009093A00380939F03011580E21807B0F44B
:104FB000C801805E9109089728F06DEF71E1011535
:104FC000110511F461EF71E1C8010E943D05802FC8
:104FD0000E94F2102696E4E00C941E3480EF898340
:104FE0008A830E94D30C8160BC0149815A8181E08F
:104FF00091E07FDDEFCFA6E0B0E0E1E0F8E20C94D5
:1050000002348C019093A00380939F03011580E2EA
:105010001807B0F4802F0E949211C801805E910998
:10502000089728F066E072E10115110511F467EFA9
:1050300071E1C8010E943D052696E4E00C941E34FF
:1050400080EF89838A830E94D30C8160BC014981EF
:105050005A8181E090E04DDDEFCFCF93DF93D82FE1
:10506000C92F97DF8D2F9C2FC6DFDF91CF91089539
:105070000F931F93CF93DF938C01862F69E474E025
:105080000E94B717892B91F4C0914904D0914A042A
:10509000209761F0F8018281833039F4CE01DDDFA1
:1050A000CE01DBDFCE01D9DF01C0E0F7DF91CF9188
:1050B0001F910F9108950F931F93CF93DF938C014E
:1050C000EB0169E474E08C2F0E94B717892B09F07B
:1050D00057C0FE01FF27D80112968C911297EB5210
:1050E000FD4F8130A9F415968C9182FD4EC080FF52
:1050F0004CC082E0808380914B0490914C040097D7
:10510000B9F48091490490914A040097C9F110C004
:105110008230A1F515968C9182FD26C080FD0AC0D3
:1051200083E0808380914D0490914E040097F1F0CC
:1051300030DF26C084E0808380914F04909150043A
:105140000097B1F78091490490914A04009701F1CA
:1051500084DF80914B0490914C04009749F7809133
:10516000490490914A04E4CF85E08083809149040A
:1051700090914A04009721F070DFF1CF86E08083A0
:10518000DF91CF911F910F91089581E08083B9CF76
:1051900080914B0490914C04B8CF0F931F93CF9301
:1051A000DF938C01EB0169E474E08C2F0E94B71748
:1051B000892B71F4DD27CB52DD4F8881F8011282F3
:1051C00018828330E9F048F4813059F0823081F060
:1051D000DF91CF911F910F9108958430B1F0853008
:1051E000B9F78091490490914A04009789F306C069
:1051F00080914B0490914C04009799F3FCDEE8CF2A
:1052000080914D0490914E04F7CF80914F0490917E
:105210005004009799F72091490430914A048091F5
:105220004B0490914C0421153105F9F2009731F7A8
:10523000C901E4CFA0E1B0E0E0E2F9E20C94F6337A
:10524000FE01319680E1DF011D928A95E9F70EE0BB
:1052500010E091E2A92E93E0B92E2FED422E512CB1
:10526000612C712C4F0173016201B1E14B165104A5
:10527000610471041CF080E1C82ED12CA601B50197
:10528000C4010E940235AC0CBD1C0D2C000CEE08B4
:10529000FF084C185D086E087F080150104019F790
:1052A0006096E0E10C9412346FEF85E290E00E948A
:1052B00011356FEF86E290E00E9411356FEF87E2C3
:1052C00090E00E94113560E088E290E00E94113584
:1052D0000E940417AFDF67E185E290E00E9411357C
:1052E00060E186E290E00E9411356FE987E290E08C
:1052F0000C9411358F929F92AF92BF92CF92DF9212
:10530000EF92FF920F93CF93DF9388E090E00E949B
:10531000F8344B015C01CFEDD4E068839982AA8216
:10532000BB821C821D821E821F8283E290E00E944B
:10533000F034282F30E040E050E060E070E080E0A2
:1053400090E000E20E942B34282939294A295B2960
:10535000288339834A835B836C837D838E839F8319
:10536000DF91CF910F91FF90EF90DF90CF90BF90A2
:10537000AF909F908F900895AAE0B0E0E2ECF9E240
:105380000C94F833FE0131968AE0DF011D928A9574
:10539000E9F796E6A92E91E0B92E8F013F01EE24A0
:1053A000E394F12C3AE7C32E31E0D32EF50181913D
:1053B0005F018F3F09F444C0F894E82FE295EF7045
:1053C000F0E021A18F70A70102C0440F551F8A95FC
:1053D000E2F7CA01922F982B91A392A1809589237D
:1053E00082A3789400C0EBE6F1E021E030E0812C6C
:1053F000912C41914F3F79F0A42FA295AF70A05E00
:10540000B0E08C9190E04F7002C0959587954A95D9
:10541000E2F780FF3BC080E090E0882A992A220FC3
:10542000331FCE16DF0629F7F50182918F3F11F069
:105430000E94520850EA5A95F1F7D8018D929C9239
:105440000E5F1F4FBBE6AB16B1E0BB0609F0AECF57
:105450004AE050E0B3018BE693E00E94CC34892B04
:10546000B9F08AE0F301ABE6B3E001900D928A95C2
:10547000E1F781E0809312020E94D30C9093110215
:10548000809310022A96EEE00C941434C901C5CF23
:10549000809112028115B1F3009110021091110256
:1054A0000E94D30C801B910B059760F34AE050E0FB
:1054B0006BE673E082E993E00E94CC34892B49F0DB
:1054C0008AE0EBE6F3E0A2E9B3E001900D928A9561
:1054D000E1F710921202D6CFCDB7DEB7AC970FB678
:1054E000F894DEBF0FBECDBF85B7806885BF85B796
:1054F000806885BF84B7877F84BF0FB6F894A8956E
:1055000080916000886180936000109260000FBEFF
:1055100080E890E00FB6F89480936100909361006A
:105520000FBE81E08093210180E598E09093E70130
:105530008093E6010E94300B0E9473170E94D90EDF
:105540000E94360F8091E20084608093E20078949C
:1055500080919E03811599F08091E9001091EC00F3
:105560008F70179511271795182B1092E9008091CD
:10557000E80083FD0E945A121F701093E90082E038
:1055800084BD93E095BD9AEF97BD80936E000E9415
:105590004316811101C088DE06E611E0D8018D9125
:1055A0008D018F3F11F00E945208B1E00B361B07AE
:1055B000A9F70BE611E0F80181918F018F3F11F0FF
:1055C0000E945208F1E00A371F07A9F78AE0E2E9D2
:1055D000F3E0DF01282F1D922A95E9F7EBE6F3E0CF
:1055E000DF011D928A95E9F780E090E00E94FD348A
:1055F000833E9E4F21F40E94431681112AC063EE20
:105600007EEF80E090E00E942B3560E082E090E049
:105610000E94113581E08093A00561E083E090E075
:105620000E94113560E074E184E090E00E942B3527
:105630000E94FD1839DE40E050E0BA018FE090E0B2
:105640000E94233540E050E0BA0183E190E00E94DF
:10565000233582E090E00E94F0348093780384E068
:1056600090E00E94FD349093A3058093A20584DE10
:10567000EFEFF6E721E0E150F0402040E1F700C015
:1056800000007ADE8091920380FF08C06FEF7FEF09
:1056900080E090E00E942B350E94D50F83E090E0DF
:1056A0000E94F0340E947C058091750381111EC018
:1056B0008FED94E01FDE8091DF04843028F40E9497
:1056C000FD188FED94E016DE0E9401091092DE04B1
:1056D0000E94480B8091DF0480FF05C060E0869542
:1056E00086950E94D01981E08093750382E191E054
:1056F0009093C6038093C50380919E03853049F43F
:1057000080919E03853009F45AC00E9419120E94AC
:10571000110C32DEB9E7AB2EB3E0BB2E12E9412EFD
:1057200013E0512ED201F501219131918D919D917E
:1057300043E0E338F40709F477C028173907A1F3E9
:10574000A2E98A2EA3E09A2E10E0D401ED90FD90FC
:105750004D01F501619071905F016E147F0449F174
:105760006E247F2400E0CC24C394D12CC3018C216F
:105770009D21892BB1F009831A830E94D30C9C834D
:105780008B83F1E0FD8391E097012C213D21232BB8
:1057900009F490E09E8349815A816B817C818D81DF
:1057A000A8D90F5FCC0CDD1C0F3001F7F501F29288
:1057B000E2921F5F153049F60E94240E3AC0809194
:1057C0009E03843021F11092760388E190E0A0E4FA
:1057D0000FB6F894A895809360000FBEA093600068
:1057E00083B7817F846083BF83B7816083BF7894F0
:1057F000889583B78E7F83BF0FB6F894A895809164
:105800006000886180936000109260000FBEB4DD7C
:10581000E2E9F3E081919191892B09F0F1C5B3E0C0
:10582000EC39FB07B9F76CCF2817390709F088CF97
:105830008EDBC090D704D090D804C114D10439F1C4
:10584000A090D904B090DA040E94D30C7C01EA182D
:10585000FB08C6010E94CC178E159F05C0F420914D
:10586000D7043091D804C9019927287F3327232BE7
:1058700009F0A0C174E0880F991F7A95E1F7895A61
:105880009B4FDC0115962C9122FF0E9439158091C7
:105890002201811511F1E0909E05F0909F05E11421
:1058A000F104D9F00E94D30C8E199F092091310583
:1058B000309132052817390780F490913405809192
:1058C0003305981709F479C167D810923105109201
:1058D000320510929E0510929F0580915304811508
:1058E00069F00E94D30C2091540430915504821B1E
:1058F000930B8F3F9F4710F40E9410128091DE049B
:10590000811509F444C08091DD04E091DF04E6953F
:10591000E695E81BE0938503853109F4ACC108F0F6
:1059200062C1893009F49DC108F050C1823009F488
:1059300086C1863009F48CC160EDE62E67E0F62E54
:105940000BE618E080918603811561F010928603C2
:105950000E94D30C90938403809383031092870357
:10596000109288030E94D30C20918303309184030A
:10597000821B930B8F3F9F4750F42E0D3F1D30939A
:1059800084032093830383E893E0F801099586E07C
:10599000E3E4F4E0DE01119601900D928A95E1F7BF
:1059A00090904404B0904504D0904604A0904704E1
:1059B000C090480410924504109246041092470487
:1059C000109248048D2D8B29811509F441C0E09077
:1059D0008B03F0908C030E94D30C9C012E193F097D
:1059E00090914104911509F406C52531310580F1E6
:1059F0009F3F19F09F5F90934104B11459F00E94AA
:105A0000C70B91E01B140CF09FEF899F802D112490
:105A100080934504D11459F00E94C70B91E01D14E6
:105A20000CF09FEF899F802D112480934604809174
:105A30004504811569F0F0904604F11449F00E9484
:105A4000B90B809345048F2D0E94B90B80934604B7
:105A50008A2D8C29811509F441C0E0908903F090CA
:105A60008A030E94D30C9C012E193F099091400497
:105A7000911509F4BBC42135310580F19F3F19F020
:105A80009F5F90934004A11459F00E94E70B91E0AE
:105A90001A140CF09FEF899F802D112480934704E6
:105AA000C11459F00E94E70B91E01C140CF09FEF19
:105AB000899F802D1124809348048091470481158B
:105AC00069F0F0904804F11449F00E94B90B8093FA
:105AD00047048F2D0E94B90B8093480480914404A1
:105AE000891119C080914504811511F08B1113C0E3
:105AF00020914604211511F02D110DC090914804FC
:105B0000911511F09C1107C030914704311103C069
:105B1000822B892B81110E94400D86E0FE01319677
:105B2000A3E4B4E001900D928A95E1F70E94110C74
:105B300090918D03891721F080938D030E94240E8C
:105B400080919E03843009F0D7CD83E08093E900F3
:105B50008091E80082FFD0CD8091E80090E085FF41
:105B600006C00E94A80E811509F48EC091E08091B4
:105B7000E8008B778093E800911509F4BDCDE090A3
:105B8000A103F090A203E981E114F10409F49BC0A0
:105B9000EE3F09F0BBC08A81833020F0855083300E
:105BA00008F0B4C0EA81EE3008F0B0C0F0E0EE5F7B
:105BB000F94C01C680E090E064CE0E9486241092E9
:105BC0009E0510929F050E94550B87CE8F3009F0DD
:105BD000B3CEE695F0E0EE56F84FE491EE2EF12CC0
:105BE00001EC19E0AFCE54EFE52EFF24F3940DEE57
:105BF0001AE0843209F4A6CE90F448E2E42EF12CA7
:105C000009E61AE0883109F49DCE833209F094CE7A
:105C1000EDE8F7E0E590F59008E419E093CE8532E1
:105C200009F08ACE8E2F63E086D5E92FF0E0E657A3
:105C3000F84FE491EE2EF12C07E418E183CEF0E06A
:105C4000E556F84FE491EE2EF12C05E819E07ACEF6
:105C5000F0E0E856F84FE491EE2EF12C06E719E05B
:105C600071CEE695F0E0EB56F84FE491EE2EF12C74
:105C700008E919E067CEF0E0E157F84FE491EE2E25
:105C8000F12C0EE11AE05ECE30E2E32EF12C9E0103
:105C90002F5F3F4F69018091E80085FD0AC0809128
:105CA000E8008B778093E8000E94A80E811599F395
:105CB0005DCF8091F100D6018D936D01B1E0EB1ABB
:105CC000F10849F753CFE43148F4E11551F0E150C0
:105CD000E33138F4F0E0E05FF94C6DC5EE3F09F4D4
:105CE00061CF8FEF898312C01A8289E08B830EC047
:105CF0008A81823081F08330B1F0813091F70E9447
:105D0000240E5FD56B837C838D839E83CE010196A9
:105D10000E94F80EF1CC88E290E062D61B821C82D1
:105D20001D828E83F3CF80919C0390919D03892BDC
:105D300069F3FE013196D2018C9111969C91B2E0EB
:105D40004B0E511C9283838332962CE9421623E03A
:105D5000520689F7DBCF8A81823019F66B817C810C
:105D60008D819E812ED588E290E05BD6CFCF4C818D
:105D70006B818A810E945E159827892798279E83C8
:105D80008D83C4CF2D813E813227232732274C813A
:105D90006B818A810E947710B9CF0E940417B6CF19
:105DA0008A81823891F1B0F48038E9F0813809F0C5
:105DB000ADCF60E08B810E94D0199B818091DF0480
:105DC00091111AC08E7F8093DF041092DE040E942E
:105DD00016099CCF833809F099CF20E04091E20466
:105DE0006C818B8106C020E04B816091E104809141
:105DF000E0040E941D198ACF81608093DF0460E077
:105E0000869586950E94D01981CF8B818093E3047B
:105E10007DCF8A818238E1F060F48038A1F081384A
:105E200009F074CF8091DF0480FF10C086958695BD
:105E30005DCF833809F06ACF8091E0048B83809135
:105E4000E1048C8363CF8091E20450CF80E04ECF99
:105E50008091E3044BCF0E9401098FED94E00E94F2
:105E6000DC1854CF80E18A8351CF1A828FED3ECF68
:105E70008C818D3108F04ACF8A809B8098248924B8
:105E80009824A12CB12CDE0111967D018D01080F03
:105E9000111D0E151F0509F439CF80E0BFED8B16DB
:105EA0009104A104B10420F4C4018F5D9C4F98D5E6
:105EB000F7018483FFEFEF1AFF0A2FEF821A920A8D
:105EC000A20AB20AE6CF80919C0390919D03892B90
:105ED00009F41CCF8C818D3108F018CF882E912CBD
:105EE000A12CB12CCA80DB80DC24CD24DC24E12C65
:105EF000F12C8E010F5F1F4F412C512C32014814A1
:105F000059046A047B0408F001CF3FEDC316D104A5
:105F1000E104F10438F4D80114966C91C6018F5D48
:105F20009C4F7FD5BFEF4B1A5B0A6B0A7B0AEFEFE2
:105F3000CE1ADE0AEE0AFE0A0F5F1F4FE0CF7AD9B3
:105F4000E5CE84E090CF8C818D3108F0DFCE882EB5
:105F5000912CA12CB12CCA80DB80DC24CD24DC2444
:105F6000E12CF12C412C512C32018E010B5F1F4F83
:105F7000481459046A047B0408F0C8CE80E0F8E5B0
:105F8000CF16F2E0DF06E104F10418F4C6018996A9
:105F900027D5D8018D938D01BFEF4B1A5B0A6B0A91
:105FA0007B0AEFEFCE1ADE0AEE0AFE0AE1CF2C8161
:105FB000022F10E02D3108F0A9CE8A819B8198270D
:105FC000892798272C01612C712C8835F2E09F07D6
:105FD00008F09CCE822E912CA12CB12C48E552E0E9
:105FE00060E070E0441955096609770942175105C8
:105FF0006105710508F48ACE20919C0330919D03C0
:10600000232B09F03EC01C0129E2220E311C80FB2B
:10601000EE24FF24E0F880FF0BC08896E1D49D8138
:1060200089279827892781159C4711F48FEF8D8345
:10603000D501C401840D951DA61DB71D80FF19C093
:10604000680141E0C41AD108CE0105968C0D9D1D52
:106050009CA78BA7C101800F911FC2D4ABA5BCA583
:106060009C9181159C4721F48FEFEBA5FCA58083C3
:106070008601FE013196EE0DFF1D2FEFE016F106B1
:1060800038F08E010F5F1F4FC12CD12C760125C037
:106090009481858181159C4711F42483258342E0F6
:1060A000E40EF11C3296EACF88E5481682E05806E5
:1060B0006104710430F4D80114966C91C201899680
:1060C000B0D4BFEFCB1ADB0AEB0AFB0AEFEF4E1A94
:1060D0005E0A6E0A7E0A0F5F1F4FC814D904EA04D5
:1060E000FB0410F313CE80919C0390919D03892BA8
:1060F00009F40CCECE0101960E94F80EFFEF21EEBE
:1061000034E0F15020403040E1F700C00000C4CA44
:1061100088E0E3E2F1E0DE01919601900D928A952C
:10612000E1F7FE0132968FE1DF011D928A95E9F7D2
:1061300086E0898388E07F96DE01159601900D92B6
:106140008A95E1F7E3CD88E6898382E08A831B8222
:106150001C82DCCD8B819C81092E000CAA0BBB0B11
:1061600025E0880F991FAA1FBB1F2A95D1F7AC0104
:10617000BD01405E5F4F6F4F7F4F481759076A0759
:106180007B0708F4C3CD8836E2E09E07A105B10580
:1061900008F0BCCD4936F2E05F076105710520F0DB
:1061A00048E652E060E070E0481B590BBC016156C4
:1061B000784FCE010196DAD3A9CD4AE150E06FEFD6
:1061C00070E0CE010796F5D380919C038983EA8223
:1061D0001B8281E08C8382E08D838DE0A2CD81E003
:1061E00090E09093A2038093A10382E390E09093C8
:1061F0009103809390030E94D30C90938F0380931C
:106200008E0384CDE114F10481F1D0909203C0900B
:10621000970300918E0310918F030E94D30C801B73
:10622000910B8536910540F1C5FE26C0D1FE24C0F4
:106230000E94D30C90938F0380938E0380919003E0
:106240009091910301979093910380939003892BF0
:1062500061F41092A2031092A10381E090E0909368
:106260009D0380939C03E12CF12C80919C038983F6
:10627000EA82809190033ACD82E390E0909391037B
:1062800080939003F2CF10929D0310929C033ECD19
:1062900040E250E06FEF70E0CE0101968AD336CD38
:1062A0008B81823009F450C078F4811136C0FE0130
:1062B00033968DE1DF011D928A95E9F788E08983A5
:1062C0008A8383E088A322CD833009F472C08430AE
:1062D00009F01CCD1C818AE0FE013596DE01919605
:1062E00001900D928A95E1F789A59AA50E94230B4A
:1062F0009AA789A78FEF183060F4FAE01F9FB001CA
:1063000011246F527D4F4AE050E0CE018196A7D311
:1063100080E089830E947317F9CC8C819AE0F92E72
:106320008E010F5D1F4FF8012F2D11922A95E9F76D
:10633000B8010E94B7178983F801DE011296019017
:106340000D92FA94E1F7E2CC1C818AE0FE013596C9
:10635000DE01919601900D928A95E1F789A19AA1AB
:106360000E94230B9AA389A38BA19CA10E94230BBB
:106370009CA38BA38DA19EA10E94230B9EA38DA302
:106380008FA198A50E94230B98A78FA38FEF183099
:1063900060F43AE0139FB00111246F577D4F4AE03B
:1063A00050E0CE0181965BD380E089830E94300B60
:1063B000ADCC2C816AE0CE018196DC01E62F1D92E6
:1063C000EA95E9F7283080F4629FB00111246F52FA
:1063D0007D4F4AE050E0F4D280E089838AE0FE01FC
:1063E000B196DE011296AACE8FEFF7CF2B30310592
:1063F00008F046CB73CB2B30310508F0FBCA28CB15
:1064000080917703811509F47BC9E0E1E9BDF2E1F0
:10641000F9BD09B400FEFDCF8091D8008F7D809337
:10642000D8008091E00082608093E0008091E000DD
:1064300081FDFCCF0E94191263C91F921FB61F92E3
:1064400011248F939F93AF93BF9380917603811113
:1064500013C08091280290912902A0912A02B09144
:106460002B024196A11DB11D809328029093290211
:10647000A0932A02B0932B02BF91AF919F918F916D
:106480001F901FBE1F90189578941F921FB61F92E1
:1064900011248F939F93AF93BF9380912802909183
:1064A0002902A0912A02B0912B020196A11DB11DD3
:1064B0008093280290932902A0932A02B0932B0282
:1064C000BF91AF919F918F911F901FBE1F90189504
:1064D0001F920F920FB60F9211242F933F934F9359
:1064E0005F936F937F938F939F93AF93BF93EF933C
:1064F000FF938091E10082FF09C08091E20082FF5A
:1065000005C08091E1008B7F8093E1008091DA00EB
:1065100080FF24C08091D80080FF20C08091DA00E5
:106520008E7F8093DA008091D90080FFA9C080E13E
:1065300089BD82E189BD09B400FEFDCF81E0809371
:106540009E0380911702811109C00E94D90E0E94FA
:10655000360F8091E20084608093E2008091E10038
:1065600080FF1AC08091E20080FF16C08091E20097
:106570008E7F8093E2008091E20080618093E20050
:106580008091D80080628093D80019BC85E0809308
:106590009E0383E0809321018091E10084FF2FC05E
:1065A0008091E20084FF2BC080E189BD82E189BD3A
:1065B00009B400FEFDCF8091D8008F7D8093D80074
:1065C0008091E1008F7E8093E1008091E2008F7ED8
:1065D0008093E2008091E20081608093E2008091EC
:1065E0001602811509F452C084E080939E038091C5
:1065F0009E03843009F052C082E080932101809193
:10660000E10083FF2CC08091E20083FF28C08091CD
:10661000E100877F8093E10082E080939E031092E7
:1066200016028091E1008E7F8093E1008091E2006C
:106630008E7F8093E2008091E20080618093E2008F
:1066400042E060E080E00E94060F8091F0008860E8
:106650008093F00081E08093210180932001FF91DD
:10666000EF91BF91AF919F918F917F916F915F91CA
:106670004F913F912F910F900FBE0F901F90189543
:1066800019BC10929E031092170268CF8091E3000C
:1066900087FF02C083E0A9CF81E0A7CF81E0ADCF23
:1066A0001F920F920FB60F921124EF92FF920F9349
:1066B0001F932F933F934F935F936F937F938F938A
:1066C0009F93AF93BF93CF93EF93FF9309EE10E0A7
:1066D000F8018081C091EC008F70C795CC27C795D9
:1066E000C82B108280EFE82EF12CF7018081877F84
:1066F000808378940E945A12F8011082F7018081F9
:1067000088608083CF70F801C083FF91EF91CF91B3
:10671000BF91AF919F918F917F916F915F914F91B9
:106720003F912F911F910F91FF90EF900F900FBE0F
:106730000F901F901895992778E0880F991F96174A
:1067400008F0961B881F7A95C9F78095089587FBF6
:10675000082E062687FD819567FD6195ECDF0EF416
:10676000919507FC81950895AA1BBB1B51E107C0B9
:10677000AA1FBB1FA617B70710F0A61BB70B881FD1
:10678000991F5A95A9F780959095BC01CD01089560
:1067900097FB072E16F4009406D077FD08D0E4DFAF
:1067A00007FC05D03EF4909581959F4F0895709514
:1067B00061957F4F0895EE0FFF1F0590F491E02D36
:1067C00009946927962769277827872778270895C6
:1067D000ABD1332312F48A1B9B0B01C0A5D1B7FFA9
:1067E0000895821B930B08952F923F924F925F92D0
:1067F0006F927F928F929F92AF92BF92CF92DF92D1
:10680000EF92FF920F931F93CF93DF93CDB7DEB735
:10681000CA1BDB0B0FB6F894DEBF0FBECDBF0994C9
:106820002A88398848885F846E847D848C849B8420
:10683000AA84B984C884DF80EE80FD800C811B812E
:10684000AA81B981CE0FD11D0FB6F894DEBF0FBE5D
:10685000CDBFED010895002E083090F0982F872FBE
:10686000762F652F542F432F322F22270850F4CF35
:10687000220F331F441F551F661F771F881F991F44
:106880000A95B2F7002D089597FD1094002E083058
:1068900098F00850232F342F452F562F672F782F2D
:1068A000892F912DF4CF15949795879577956795B6
:1068B00057954795379527950A95AAF71124002DE6
:1068C00008958F929F92AF92BF92CF92DF92EF92F4
:1068D000FF92CF93DF93EC01688179818A819B815C
:1068E000611571058105910521F464E279ED8BE56F
:1068F00097E02DE133EF41E050E0C8D049015A0163
:106900009B01AC01A7EAB1E4DDD06B017C01ACEEE8
:10691000B4EFA5019401E2D0DC01CB018C0D9D1DEB
:10692000AE1DBF1DB7FF03C00197A109B048888302
:106930009983AA83BB839F77DF91CF91FF90EF90DC
:10694000DF90CF90BF90AF909F908F900895B9CF78
:1069500080E091E0B6CFA0E0B0E08093000190939A
:106960000101A0930201B09303010895FB01DC0132
:1069700002C005900D9241505040D8F70895FC0197
:106980004150504030F001900616D1F73197CF01B9
:106990000895882799270895FB01DC0104C08D9193
:1069A0000190801921F441505040C8F7881B990B81
:1069B0000895DC0101C06D9341505040E0F7089507
:1069C000DC01CB01FC01F999FECF06C0F2BDE1BDAF
:1069D000F89A319600B40D9241505040B8F708959E
:1069E000F999FECF92BD81BDF89A992780B5089597
:1069F000A6E1B0E044E050E0E5CFA8E1B0E042E03D
:106A000050E0E0CFDC01A40FB51F4150504040F0F2
:106A1000CB01840F951F2E9105D041505040D8F7DF
:106A20000895262FF999FECF92BD81BDF89A01975E
:106A300000B4021639F01FBA20BD0FB6F894FA9AC6
:106A4000F99A0FBE08950396272FECDFEADF252F72
:106A5000E9DF242FE7CF0196272FE4DFE2CFDC0127
:106A6000CB0102C02D9105D041505040D8F7089578
:106A7000262FF999FECF1FBA92BD81BD20BD0FB65A
:106A8000F894FA9AF99A0FBE01960895052E97FB8D
:106A900016F400940FD057FD05D024D007FC02D087
:106AA00046F408C050954095309521953F4F4F4F83
:106AB0005F4F089590958095709561957F4F8F4FAA
:106AC0009F4F089531D0A59F900DB49F900DA49F26
:106AD000800D911D11240895B7FFF4CFF3DF821BC1
:106AE000930B0895A1E21A2EAA1BBB1BFD010DC03A
:106AF000AA1FBB1FEE1FFF1FA217B307E407F5076E
:106B000020F0A21BB30BE40BF50B661F771F881F49
:106B1000991F1A9469F760957095809590959B01DF
:106B2000AC01BD01CF010895A29FB001B39FC00188
:106B3000A39F700D811D1124911DB29F700D811DA9
:106B40001124911D0895F894FFCF750D7A0D7C0DD9
:106B5000810D910D910D910D910D910D910D910D55
:106B6000910D830D870D8A0D8F0D9F0DA50DA90D1C
:106B700037135D1363135D136313B513D6136313D8
:106B8000DC14E914C81D301ED01D9A1D9E1DD41D95
:106B9000A21DD81DE41DAE1D291EB21DE81DB61D87
:106BA000EC1D111EBA1DF01D181EC01DF61DFE1D88
:106BB000A61DDC1DAA1DE01DC41DFA1D081E211EF8
:106BC000271E941DCC1D371E661D6C1D541D5C1D9B
:106BD000721D781D7E1D571E6E1E721E761E7A1E39
:106BE0007E1E821E861E8A1E8E1E921EEC1FEC1FAB
:106BF00023202320D320EE2047204720F3206621A6
:106C0000772177218830A330AA30862E862EDD307A
:106C1000EF30023143314831862E862E862E503198
:106C2000742E782EAB2EB72EC22ECD2ED02E092F3D
:106C30002B2F712E7330322F352F382F632F9F2F2C
:066C4000A12FA32FD72FA6
:106C46000100000001010201191A1B1C1D1E1F2054
:106C56002122D00C3B10511056105B103210000050
:106C6600010001D7DF5A8551BF42F5004422B684A0
:106C7600016201AC008A02A302C302000102020201
:106C8600020606060909090909090F0F0F0F0F0F5A
:106C96001515151819191919191919191919232456
:106CA6002525252525253132676636C6F0F1F4F50A
:106CB600F6F73534979694959392E200E900EA0048
:106CC600B500B600B700CD008301CC008A01920161
:106CD60094012102230224022502260227022A0207
:106CE600B300B4006F0070009F01CB019F02A002A9
:106CF600E200E900EA00B500B600B700CD00830166
:106D0600CC008A0192019401210223022402250269
:106D1600260227022A02B300B4006F0070009F010A
:066D2600CB019F02A00258
:00000001FF
